 ZLib

 Timestamp is 54e2a5a7 (Mon Feb 16 20:21:27 2015)

 Preferred load address is 10000000

 Start         Length     Name                   Class
 0001:00000000 00007352H .text                   CODE
 0001:00007352 0000000aH .text$x                 CODE
 0001:0000735c 000000d0H .text$yc                CODE
 0001:0000742c 00000084H .text$yd                CODE
 0002:00000000 00000114H .idata$5                DATA
 0002:00000114 00000004H .CRT$XCA                DATA
 0002:00000118 00000014H .CRT$XCU                DATA
 0002:0000012c 00000004H .CRT$XCZ                DATA
 0002:00000130 00000004H .CRT$XIA                DATA
 0002:00000134 00000004H .CRT$XIAA               DATA
 0002:00000138 00000004H .CRT$XIC                DATA
 0002:0000013c 00000004H .CRT$XIZ                DATA
 0002:00000140 000017b8H .rdata                  DATA
 0002:000018f8 00000068H .rdata$debug            DATA
 0002:00001960 0000017cH .rdata$r                DATA
 0002:00001ae0 00000008H .rdata$sxdata           DATA
 0002:00001ae8 00000004H .rtc$IAA                DATA
 0002:00001aec 00000004H .rtc$IZZ                DATA
 0002:00001af0 00000004H .rtc$TAA                DATA
 0002:00001af4 00000004H .rtc$TZZ                DATA
 0002:00001af8 00000134H .xdata$x                DATA
 0002:00001c2c 00000050H .idata$2                DATA
 0002:00001c7c 00000014H .idata$3                DATA
 0002:00001c90 00000114H .idata$4                DATA
 0002:00001da4 000004c2H .idata$6                DATA
 0002:00002270 00000535H .edata                  DATA
 0003:00000000 0000129cH .data                   DATA
 0003:000012a0 0000035cH .bss                    DATA
 0004:00000000 00000058H .rsrc$01                DATA
 0004:00000060 00000180H .rsrc$02                DATA

  Address         Publics by Value              Rva+Base       Lib:Object

 0000:00000002       ___safe_se_handler_count   00000002     <absolute>
 0000:00000000       ___ImageBase               10000000     <linker-defined>
 0001:00000000       ??$_Allocate@D@std@@YGPADIPAD@Z 10001000 f i ZLibInit.obj
 0001:00000027       ??$addressof@D@std@@YGPADAAD@Z 10001027 f i ZLibInit.obj
 0001:0000002e       ??$construct@PADAAPAD@?$_Wrap_alloc@V?$allocator@D@std@@@std@@QAEXPAPADAAPAD@Z 1000102e f i ZLibInit.obj
 0001:00000041       ??$construct@PADAAPAD@?$allocator@D@std@@QAEXPAPADAAPAD@Z 10001041 f i ZLibInit.obj
 0001:00000054       ??$construct@PADAAPAD@?$allocator_traits@V?$allocator@D@std@@@std@@SGXAAV?$allocator@D@1@PAPADAAPAD@Z 10001054 f i ZLibInit.obj
 0001:00000067       ??$destroy@PAD@?$_Wrap_alloc@V?$allocator@D@std@@@std@@QAEXPAPAD@Z 10001067 f i ZLibInit.obj
 0001:0000006a       ??$destroy@PAD@?$allocator@D@std@@QAEXPAPAD@Z 1000106a f i ZLibInit.obj
 0001:0000006d       ??$destroy@PAD@?$allocator_traits@V?$allocator@D@std@@@std@@SGXAAV?$allocator@D@1@PAPAD@Z 1000106d f i ZLibInit.obj
 0001:00000070       ??$forward@AAPAD@std@@YGAAPADAAPAD@Z 10001070 f i ZLibInit.obj
 0001:00000077       ??0?$_String_alloc@$0A@U?$_String_base_types@DV?$allocator@D@std@@@std@@@std@@QAE@ABV?$allocator@D@1@@Z 10001077 f i ZLibInit.obj
 0001:00000084       ??0?$_String_val@U?$_Simple_types@D@std@@@std@@QAE@XZ 10001084 f i ZLibInit.obj
 0001:0000008f       ??0?$_Wrap_alloc@V?$allocator@D@std@@@std@@QAE@XZ 1000108f f i ZLibInit.obj
 0001:00000092       ??0?$allocator@D@std@@QAE@XZ 10001092 f i ZLibInit.obj
 0001:00000095       ??0?$basic_string@DU?$char_traits@D@std@@V?$allocator@D@2@@std@@QAE@PBD@Z 10001095 f i ZLibInit.obj
 0001:000000c2       ??0_Generic_error_category@std@@QAE@XZ 100010c2 f i ZLibInit.obj
 0001:000000cb       ??0_Iostream_error_category@std@@QAE@XZ 100010cb f i ZLibInit.obj
 0001:000000d4       ??0_System_error_category@std@@QAE@XZ 100010d4 f i ZLibInit.obj
 0001:000000dd       ??0error_category@std@@QAE@XZ 100010dd f i ZLibInit.obj
 0001:000000e6       ??0error_condition@std@@QAE@HABVerror_category@1@@Z 100010e6 f i ZLibInit.obj
 0001:000000f8       ??1?$basic_string@DU?$char_traits@D@std@@V?$allocator@D@2@@std@@QAE@XZ 100010f8 f i ZLibInit.obj
 0001:00000119       ??1_Generic_error_category@std@@UAE@XZ 10001119 f i ZLibInit.obj
 0001:00000120       ??1_Iostream_error_category@std@@UAE@XZ 10001120 f i ZLibInit.obj
 0001:00000127       ??1_System_error_category@std@@UAE@XZ 10001127 f i ZLibInit.obj
 0001:0000012e       ??1error_category@std@@UAE@XZ 1000112e f i ZLibInit.obj
 0001:00000135       ??2@YAPAXIPAX@Z            10001135 f i ZLibInit.obj
 0001:0000013a       ??3@YAXPAX0@Z              1000113a f i ZLibInit.obj
 0001:0000013b       ??8error_category@std@@QBE_NABV01@@Z 1000113b f i ZLibInit.obj
 0001:00000147       ??8error_condition@std@@QBE_NABV01@@Z 10001147 f i ZLibInit.obj
 0001:00000163       ??_E_Generic_error_category@std@@UAEPAXI@Z 10001163 f i ZLibInit.obj
 0001:00000163       ??_G_Generic_error_category@std@@UAEPAXI@Z 10001163 f i ZLibInit.obj
 0001:00000180       ??_G_Iostream_error_category@std@@UAEPAXI@Z 10001180 f i ZLibInit.obj
 0001:00000180       ??_E_Iostream_error_category@std@@UAEPAXI@Z 10001180 f i ZLibInit.obj
 0001:0000019d       ??_E_System_error_category@std@@UAEPAXI@Z 1000119d f i ZLibInit.obj
 0001:0000019d       ??_G_System_error_category@std@@UAEPAXI@Z 1000119d f i ZLibInit.obj
 0001:000001ba       ??_Eerror_category@std@@UAEPAXI@Z 100011ba f i ZLibInit.obj
 0001:000001ba       ??_Gerror_category@std@@UAEPAXI@Z 100011ba f i ZLibInit.obj
 0001:000001d7       ?_Copy@?$basic_string@DU?$char_traits@D@std@@V?$allocator@D@2@@std@@QAEXII@Z 100011d7 f i ZLibInit.obj
 0001:000002ec       ?_Eos@?$basic_string@DU?$char_traits@D@std@@V?$allocator@D@2@@std@@QAEXI@Z 100012ec f i ZLibInit.obj
 0001:00000302       ?_Getal@?$_String_alloc@$0A@U?$_String_base_types@DV?$allocator@D@std@@@std@@@std@@QBE?AU?$_Wrap_alloc@V?$allocator@D@std@@@2@XZ 10001302 f i ZLibInit.obj
 0001:00000309       ?_Grow@?$basic_string@DU?$char_traits@D@std@@V?$allocator@D@2@@std@@QAE_NI_N@Z 10001309 f i ZLibInit.obj
 0001:0000036a       ?_Inside@?$basic_string@DU?$char_traits@D@std@@V?$allocator@D@2@@std@@QAE_NPBD@Z 1000136a f i ZLibInit.obj
 0001:000003a2       ?_Myptr@?$_String_val@U?$_Simple_types@D@std@@@std@@QAEPADXZ 100013a2 f i ZLibInit.obj
 0001:000003ad       ?_Myptr@?$_String_val@U?$_Simple_types@D@std@@@std@@QBEPBDXZ 100013ad f i ZLibInit.obj
 0001:000003b8       ?_Tidy@?$basic_string@DU?$char_traits@D@std@@V?$allocator@D@2@@std@@QAEX_NI@Z 100013b8 f i ZLibInit.obj
 0001:000003fa       ?_Xlen@?$basic_string@DU?$char_traits@D@std@@V?$allocator@D@2@@std@@QBEXXZ 100013fa f i ZLibInit.obj
 0001:00000406       ?_Xran@?$basic_string@DU?$char_traits@D@std@@V?$allocator@D@2@@std@@QBEXXZ 10001406 f i ZLibInit.obj
 0001:00000412       ?allocate@?$_Wrap_alloc@V?$allocator@D@std@@@std@@QAEPADI@Z 10001412 f i ZLibInit.obj
 0001:00000420       ?allocate@?$allocator@D@std@@QAEPADI@Z 10001420 f i ZLibInit.obj
 0001:0000042e       ?assign@?$basic_string@DU?$char_traits@D@std@@V?$allocator@D@2@@std@@QAEAAV12@ABV12@II@Z 1000142e f i ZLibInit.obj
 0001:000004c0       ?assign@?$basic_string@DU?$char_traits@D@std@@V?$allocator@D@2@@std@@QAEAAV12@PBD@Z 100014c0 f i ZLibInit.obj
 0001:000004dd       ?assign@?$basic_string@DU?$char_traits@D@std@@V?$allocator@D@2@@std@@QAEAAV12@PBDI@Z 100014dd f i ZLibInit.obj
 0001:00000555       ?assign@?$char_traits@D@std@@SAXAADABD@Z 10001555 f i ZLibInit.obj
 0001:00000562       ?category@error_code@std@@QBEABVerror_category@2@XZ 10001562 f i ZLibInit.obj
 0001:00000566       ?category@error_condition@std@@QBEABVerror_category@2@XZ 10001566 f i ZLibInit.obj
 0001:0000056a       ?copy@?$char_traits@D@std@@SAPADPADPBDI@Z 1000156a f i ZLibInit.obj
 0001:0000057e       ?deallocate@?$_Wrap_alloc@V?$allocator@D@std@@@std@@QAEXPADI@Z 1000157e f i ZLibInit.obj
 0001:0000058b       ?deallocate@?$allocator@D@std@@QAEXPADI@Z 1000158b f i ZLibInit.obj
 0001:00000598       ?default_error_condition@_System_error_category@std@@UBE?AVerror_condition@2@H@Z 10001598 f i ZLibInit.obj
 0001:000005c3       ?default_error_condition@error_category@std@@UBE?AVerror_condition@2@H@Z 100015c3 f i ZLibInit.obj
 0001:000005d3       ?equivalent@error_category@std@@UBE_NABVerror_code@2@H@Z 100015d3 f i ZLibInit.obj
 0001:000005ee       ?equivalent@error_category@std@@UBE_NHABVerror_condition@2@@Z 100015ee f i ZLibInit.obj
 0001:0000060d       ?erase@?$basic_string@DU?$char_traits@D@std@@V?$allocator@D@2@@std@@QAEAAV12@I@Z 1000160d f i ZLibInit.obj
 0001:00000639       ?erase@?$basic_string@DU?$char_traits@D@std@@V?$allocator@D@2@@std@@QAEAAV12@II@Z 10001639 f i ZLibInit.obj
 0001:000006ba       ?generic_category@std@@YGABVerror_category@1@XZ 100016ba f i ZLibInit.obj
 0001:000006c0       ?length@?$char_traits@D@std@@SAIPBD@Z 100016c0 f i ZLibInit.obj
 0001:000006d4       ?max_size@?$_Wrap_alloc@V?$allocator@D@std@@@std@@QBEIXZ 100016d4 f i ZLibInit.obj
 0001:000006d8       ?max_size@?$allocator@D@std@@QBEIXZ 100016d8 f i ZLibInit.obj
 0001:000006dc       ?max_size@?$allocator_traits@V?$allocator@D@std@@@std@@SGIABV?$allocator@D@2@@Z 100016dc f i ZLibInit.obj
 0001:000006e2       ?max_size@?$basic_string@DU?$char_traits@D@std@@V?$allocator@D@2@@std@@QBEIXZ 100016e2 f i ZLibInit.obj
 0001:000006e6       ?message@_Generic_error_category@std@@UBE?AV?$basic_string@DU?$char_traits@D@std@@V?$allocator@D@2@@2@H@Z 100016e6 f i ZLibInit.obj
 0001:00000712       ?message@_Iostream_error_category@std@@UBE?AV?$basic_string@DU?$char_traits@D@std@@V?$allocator@D@2@@2@H@Z 10001712 f i ZLibInit.obj
 0001:00000741       ?message@_System_error_category@std@@UBE?AV?$basic_string@DU?$char_traits@D@std@@V?$allocator@D@2@@2@H@Z 10001741 f i ZLibInit.obj
 0001:0000076d       ?move@?$char_traits@D@std@@SAPADPADPBDI@Z 1000176d f i ZLibInit.obj
 0001:00000782       ?name@_Generic_error_category@std@@UBEPBDXZ 10001782 f i ZLibInit.obj
 0001:00000788       ?name@_Iostream_error_category@std@@UBEPBDXZ 10001788 f i ZLibInit.obj
 0001:0000078e       ?name@_System_error_category@std@@UBEPBDXZ 1000178e f i ZLibInit.obj
 0001:00000794       ?size@?$basic_string@DU?$char_traits@D@std@@V?$allocator@D@2@@std@@QBEIXZ 10001794 f i ZLibInit.obj
 0001:00000798       ?system_category@std@@YGABVerror_category@1@XZ 10001798 f i ZLibInit.obj
 0001:0000079e       ?value@error_code@std@@QBEHXZ 1000179e f i ZLibInit.obj
 0001:000007a1       ?value@error_condition@std@@QBEHXZ 100017a1 f i ZLibInit.obj
 0001:000007a4       _DllMain@12                100017a4 f   ZLibInit.obj
 0001:000007d1       _adler32@12                100017d1 f   adler32.obj
 0001:000008e9       _compress2@20              100018e9 f   compress.obj
 0001:00000968       _compress@16               10001968 f   compress.obj
 0001:00000982       _crc32@12                  10001982 f   crc32.obj
 0001:00000a70       _get_crc_table@0           10001a70 f   crc32.obj
 0001:000011ee       _deflate@8                 100021ee f   deflate.obj
 0001:00001424       _deflateCopy@8             10002424 f   deflate.obj
 0001:0000158c       _deflateEnd@4              1000258c f   deflate.obj
 0001:00001619       _deflateInit2_@32          10002619 f   deflate.obj
 0001:000017d5       _deflateInit_@16           100027d5 f   deflate.obj
 0001:000017f5       _deflateParams@12          100027f5 f   deflate.obj
 0001:0000189f       _deflateReset@4            1000289f f   deflate.obj
 0001:0000190e       _deflateSetDictionary@12   1000290e f   deflate.obj
 0001:000022dc       _gzclose@4                 100032dc f   gzio.obj
 0001:0000231c       _gzdopen@8                 1000331c f   gzio.obj
 0001:00002354       _gzeof@4                   10003354 f   gzio.obj
 0001:0000236c       _gzerror@8                 1000336c f   gzio.obj
 0001:00002415       _gzflush@8                 10003415 f   gzio.obj
 0001:00002441       _gzgetc@4                  10003441 f   gzio.obj
 0001:00002466       _gzgets@12                 10003466 f   gzio.obj
 0001:000024b0       _gzopen@8                  100034b0 f   gzio.obj
 0001:000024c2       _gzprintf                  100034c2 f   gzio.obj
 0001:0000250c       _gzputc@8                  1000350c f   gzio.obj
 0001:00002536       _gzputs@8                  10003536 f   gzio.obj
 0001:00002551       _gzread@12                 10003551 f   gzio.obj
 0001:00002711       _gzrewind@4                10003711 f   gzio.obj
 0001:0000276f       _gzseek@12                 1000376f f   gzio.obj
 0001:0000289c       _gzsetparams@12            1000389c f   gzio.obj
 0001:000028f0       _gztell@4                  100038f0 f   gzio.obj
 0001:00002900       _gzwrite@12                10003900 f   gzio.obj
 0001:000029a9       _inflate_blocks@12         100039a9 f   infblock.obj
 0001:00003249       _inflate_blocks_free@8     10004249 f   infblock.obj
 0001:0000327c       _inflate_blocks_new@12     1000427c f   infblock.obj
 0001:000032fc       _inflate_blocks_reset@12   100042fc f   infblock.obj
 0001:0000335e       _inflate_blocks_sync_point@4 1000435e f   infblock.obj
 0001:0000336d       _inflate_set_dictionary@12 1000436d f   infblock.obj
 0001:00003397       _inflate_codes@12          10004397 f   infcodes.obj
 0001:000039e7       _inflate_codes_free@8      100049e7 f   infcodes.obj
 0001:000039f8       _inflate_codes_new@20      100049f8 f   infcodes.obj
 0001:00003a2f       _inflate_fast@24           10004a2f f   inffast.obj
 0001:00003d6c       _inflate@8                 10004d6c f   inflate.obj
 0001:000040c8       _inflateEnd@4              100050c8 f   inflate.obj
 0001:00004105       _inflateInit2_@16          10005105 f   inflate.obj
 0001:000041dd       _inflateInit_@12           100051dd f   inflate.obj
 0001:000041f3       _inflateReset@4            100051f3 f   inflate.obj
 0001:00004232       _inflateSetDictionary@12   10005232 f   inflate.obj
 0001:000042a1       _inflateSync@4             100052a1 f   inflate.obj
 0001:0000433f       _inflateSyncPoint@4        1000533f f   inflate.obj
 0001:000047c0       _inflate_trees_bits@20     100057c0 f   inftrees.obj
 0001:0000483c       _inflate_trees_dynamic@36  1000583c f   inftrees.obj
 0001:00004950       _inflate_trees_fixed@20    10005950 f   inftrees.obj
 0001:0000497f       _inflate_flush@12          1000597f f   infutil.obj
 0001:00004a75       __tr_align@4               10005a75 f   trees.obj
 0001:00004c29       __tr_flush_block@16        10005c29 f   trees.obj
 0001:00004de2       __tr_init@4                10005de2 f   trees.obj
 0001:00004e4a       __tr_stored_block@16       10005e4a f   trees.obj
 0001:00004ed5       __tr_tally@12              10005ed5 f   trees.obj
 0001:00006313       _uncompress@16             10007313 f   uncompr.obj
 0001:0000638c       _zError@4                  1000738c f   zutil.obj
 0001:0000639f       _zcalloc@12                1000739f f   zutil.obj
 0001:000063b2       _zcfree@8                  100073b2 f   zutil.obj
 0001:000063c0       _zlibVersion@0             100073c0 f   zutil.obj
 0001:000063c6       ??0CompressionStream@@QAE@W4Mode@0@@Z 100073c6 f   Compression1.obj
 0001:00006438       ??1CompressionStream@@QAE@XZ 10007438 f   Compression1.obj
 0001:00006463       ?ReadCompressed@CompressionStream@@QAEKPAXK@Z 10007463 f   Compression1.obj
 0001:000064cf       ?ReadExpanded@CompressionStream@@QAEKPAXK@Z 100074cf f   Compression1.obj
 0001:00006531       ?SetCompressInput@CompressionStream@@QAEXPBXI_N@Z 10007531 f   Compression1.obj
 0001:00006555       ?SetExpandInput@CompressionStream@@QAEXPBXI@Z 10007555 f   Compression1.obj
 0001:00006570       ?ZLibMemAlloc@@YGPAXPAXII@Z 10007570 f   CompressionMem1.obj
 0001:00006589       ?ZLibMemFree@@YGXPAX0@Z    10007589 f   CompressionMem1.obj
 0001:0000659c       ?ZLibMemInitialize@@YGXXZ  1000759c f   CompressionMem1.obj
 0001:000065b2       ?ZLibMemShutdown@@YGXXZ    100075b2 f   CompressionMem1.obj
 0001:000065c6       _DisableThreadLibraryCalls@4 100075c6 f   kernel32:KERNEL32.dll
 0001:000065cc       _GetModuleHandleA@4        100075cc f   kernel32:KERNEL32.dll
 0001:000065d2       ?MemPoolCreate@@YGPAU_HMEMPOOL@@PBDI@Z 100075d2 f   Memory:Memory.dll
 0001:000065d8       ?MemPoolDestroy@@YGXPAU_HMEMPOOL@@@Z 100075d8 f   Memory:Memory.dll
 0001:000065de       ?MemPoolAlloc@@YGPAXPAU_HMEMPOOL@@I@Z 100075de f   Memory:Memory.dll
 0001:000065e4       ?MemPoolFree@@YGXPAU_HMEMPOOL@@PAX@Z 100075e4 f   Memory:Memory.dll
 0001:000065ea       ?_Xbad_alloc@std@@YAXXZ    100075ea f   msvcprt:MSVCP110.dll
 0001:000065f0       ?_Xlength_error@std@@YAXPBD@Z 100075f0 f   msvcprt:MSVCP110.dll
 0001:000065f6       ?_Xout_of_range@std@@YAXPBD@Z 100075f6 f   msvcprt:MSVCP110.dll
 0001:000065fc       ?_Syserror_map@std@@YAPBDH@Z 100075fc f   msvcprt:MSVCP110.dll
 0001:00006602       ?_Winerror_map@std@@YAPBDH@Z 10007602 f   msvcprt:MSVCP110.dll
 0001:00006608       __purecall                 10007608 f   MSVCRT:MSVCR110.dll
 0001:0000660e       ??2@YAPAXI@Z               1000760e f   MSVCRT:MSVCR110.dll
 0001:00006614       ??3@YAXPAX@Z               10007614 f   MSVCRT:MSVCR110.dll
 0001:0000661a       ___atonexitinit            1000761a f   MSVCRT:atonexit.obj
 0001:00006656       __onexit                   10007656 f   MSVCRT:atonexit.obj
 0001:000066fb       _atexit                    100076fb f   MSVCRT:atonexit.obj
 0001:00006710       _memcpy                    10007710 f   MSVCRT:MSVCR110.dll
 0001:00006716       _strlen                    10007716 f   MSVCRT:MSVCR110.dll
 0001:0000671c       _memmove                   1000771c f   MSVCRT:MSVCR110.dll
 0001:00006722       __CxxThrowException@8      10007722 f   MSVCRT:MSVCR110.dll
 0001:00006728       __EH_prolog                10007728 f   MSVCRT:ehprolog.obj
 0001:00006748       ___CxxFrameHandler3        10007748 f   MSVCRT:MSVCR110.dll
 0001:0000674e       ??0type_info@@AAE@ABV0@@Z  1000774e f   MSVCRT:ti_inst.obj
 0001:00006759       ??4type_info@@AAEAAV0@ABV0@@Z 10007759 f   MSVCRT:ti_inst.obj
 0001:0000675e       ??_Etype_info@@UAEPAXI@Z   1000775e f i MSVCRT:ti_inst.obj
 0001:000067a8       _memset                    100077a8 f   MSVCRT:MSVCR110.dll
 0001:000067ae       _fclose                    100077ae f   MSVCRT:MSVCR110.dll
 0001:000067b4       __fdopen                   100077b4 f   MSVCRT:MSVCR110.dll
 0001:000067ba       _ferror                    100077ba f   MSVCRT:MSVCR110.dll
 0001:000067c0       _fflush                    100077c0 f   MSVCRT:MSVCR110.dll
 0001:000067c6       _fopen                     100077c6 f   MSVCRT:MSVCR110.dll
 0001:000067cc       _fprintf                   100077cc f   MSVCRT:MSVCR110.dll
 0001:000067d2       _fputc                     100077d2 f   MSVCRT:MSVCR110.dll
 0001:000067d8       _fread                     100077d8 f   MSVCRT:MSVCR110.dll
 0001:000067de       _fseek                     100077de f   MSVCRT:MSVCR110.dll
 0001:000067e4       _ftell                     100077e4 f   MSVCRT:MSVCR110.dll
 0001:000067ea       _fwrite                    100077ea f   MSVCRT:MSVCR110.dll
 0001:000067f0       _rewind                    100077f0 f   MSVCRT:MSVCR110.dll
 0001:000067f6       _sprintf                   100077f6 f   MSVCRT:MSVCR110.dll
 0001:000067fc       _vsprintf                  100077fc f   MSVCRT:MSVCR110.dll
 0001:00006802       _strcpy                    10007802 f   MSVCRT:MSVCR110.dll
 0001:00006808       _strcat                    10007808 f   MSVCRT:MSVCR110.dll
 0001:0000680e       __errno                    1000780e f   MSVCRT:MSVCR110.dll
 0001:00006814       _free                      10007814 f   MSVCRT:MSVCR110.dll
 0001:0000681a       _malloc                    1000781a f   MSVCRT:MSVCR110.dll
 0001:00006820       __alloca_probe             10007820     MSVCRT:chkstk.obj
 0001:00006820       __chkstk                   10007820 f   MSVCRT:chkstk.obj
 0001:0000684c       _calloc                    1000784c f   MSVCRT:MSVCR110.dll
 0001:0000689e       _NtCurrentTeb              1000789e f i MSVCRT:crtdll.obj
 0001:000068a5       __CRT_INIT@12              100078a5 f   MSVCRT:crtdll.obj
 0001:00006a9a       __DllMainCRTStartup@12     10007a9a f   MSVCRT:crtdll.obj
 0001:00006bf0       __lock                     10007bf0 f   MSVCRT:MSVCR110.dll
 0001:00006bf6       __unlock                   10007bf6 f   MSVCRT:MSVCR110.dll
 0001:00006bfc       __calloc_crt               10007bfc f   MSVCRT:MSVCR110.dll
 0001:00006c02       ___dllonexit               10007c02 f   MSVCRT:MSVCR110.dll
 0001:00006c10       __SEH_prolog4              10007c10 f   MSVCRT:sehprolg4.obj
 0001:00006c55       __SEH_epilog4              10007c55 f   MSVCRT:sehprolg4.obj
 0001:00006c69       __except_handler4          10007c69 f   MSVCRT:chandler4gs.obj
 0001:00006c8c       ??_M@YGXPAXIHP6EX0@Z@Z     10007c8c f   MSVCRT:ehvecdtr.obj
 0001:00006d14       ?__ArrayUnwind@@YGXPAXIHP6EX0@Z@Z 10007d14 f   MSVCRT:ehvecdtr.obj
 0001:00006d72       ??1type_info@@UAE@XZ       10007d72 f   MSVCRT:MSVCR110.dll
 0001:00006d78       ___CppXcptFilter           10007d78 f   MSVCRT:MSVCR110.dll
 0001:00006d7e       __amsg_exit                10007d7e f   MSVCRT:MSVCR110.dll
 0001:00006d90       __FindPESection            10007d90 f   MSVCRT:pesect.obj
 0001:00006de0       __IsNonwritableInCurrentImage 10007de0 f   MSVCRT:pesect.obj
 0001:00006ea0       __ValidateImageBase        10007ea0 f   MSVCRT:pesect.obj
 0001:00006ed1       ___security_init_cookie    10007ed1 f   MSVCRT:gs_support.obj
 0001:00006f6c       __malloc_crt               10007f6c f   MSVCRT:MSVCR110.dll
 0001:00006f72       __RTC_Initialize           10007f72 f   MSVCRT:initsect.obj
 0001:00006f92       __RTC_Terminate            10007f92 f   MSVCRT:initsect.obj
 0001:00006fb2       __initterm                 10007fb2 f   MSVCRT:MSVCR110.dll
 0001:00006fb8       __initterm_e               10007fb8 f   MSVCRT:MSVCR110.dll
 0001:00006fbe       ___clean_type_info_names   10007fbe f   MSVCRT:tncleanup.obj
 0001:00006fca       @__security_check_cookie@4 10007fca f   MSVCRT:secchk.obj
 0001:00006fda       __except_handler4_common   10007fda f   MSVCRT:MSVCR110.dll
 0001:00006fe0       ?terminate@@YAXXZ          10007fe0 f   MSVCRT:MSVCR110.dll
 0001:00006fe6       ___clean_type_info_names_internal 10007fe6 f   MSVCRT:MSVCR110.dll
 0001:00006fec       ___raise_securityfailure   10007fec f   MSVCRT:gs_report.obj
 0001:00007029       ___report_gsfailure        10008029 f   MSVCRT:gs_report.obj
 0001:00007122       ___report_rangecheckfailure 10008122 f   MSVCRT:gs_report.obj
 0001:0000712e       ___report_securityfailure  1000812e f   MSVCRT:gs_report.obj
 0001:000071fc       ___report_securityfailureEx 100081fc f   MSVCRT:gs_report.obj
 0001:00007310       __crt_debugger_hook        10008310 f   MSVCRT:MSVCR110.dll
 0001:00007316       ___crtUnhandledException   10008316 f   MSVCRT:MSVCR110.dll
 0001:0000731c       ___crtTerminateProcess     1000831c f   MSVCRT:MSVCR110.dll
 0001:00007322       _EncodePointer@4           10008322 f   kernel32:KERNEL32.dll
 0001:00007328       _DecodePointer@4           10008328 f   kernel32:KERNEL32.dll
 0001:0000732e       _QueryPerformanceCounter@4 1000832e f   kernel32:KERNEL32.dll
 0001:00007334       _GetCurrentProcessId@0     10008334 f   kernel32:KERNEL32.dll
 0001:0000733a       _GetCurrentThreadId@0      1000833a f   kernel32:KERNEL32.dll
 0001:00007340       _GetSystemTimeAsFileTime@4 10008340 f   kernel32:KERNEL32.dll
 0001:00007346       _IsDebuggerPresent@0       10008346 f   kernel32:KERNEL32.dll
 0001:0000734c       _IsProcessorFeaturePresent@4 1000834c f   kernel32:KERNEL32.dll
 0002:00000000       __imp__DisableThreadLibraryCalls@4 10009000     kernel32:KERNEL32.dll
 0002:00000004       __imp__GetModuleHandleA@4  10009004     kernel32:KERNEL32.dll
 0002:00000008       __imp__IsDebuggerPresent@0 10009008     kernel32:KERNEL32.dll
 0002:0000000c       __imp__GetSystemTimeAsFileTime@4 1000900c     kernel32:KERNEL32.dll
 0002:00000010       __imp__GetCurrentThreadId@0 10009010     kernel32:KERNEL32.dll
 0002:00000014       __imp__GetCurrentProcessId@0 10009014     kernel32:KERNEL32.dll
 0002:00000018       __imp__QueryPerformanceCounter@4 10009018     kernel32:KERNEL32.dll
 0002:0000001c       __imp__DecodePointer@4     1000901c     kernel32:KERNEL32.dll
 0002:00000020       __imp__EncodePointer@4     10009020     kernel32:KERNEL32.dll
 0002:00000024       __imp__IsProcessorFeaturePresent@4 10009024     kernel32:KERNEL32.dll
 0002:00000028       \177KERNEL32_NULL_THUNK_DATA 10009028     kernel32:KERNEL32.dll
 0002:0000002c       __imp_?_Syserror_map@std@@YAPBDH@Z 1000902c     msvcprt:MSVCP110.dll
 0002:00000030       __imp_?_Winerror_map@std@@YAPBDH@Z 10009030     msvcprt:MSVCP110.dll
 0002:00000034       __imp_?_Xlength_error@std@@YAXPBD@Z 10009034     msvcprt:MSVCP110.dll
 0002:00000038       __imp_?_Xbad_alloc@std@@YAXXZ 10009038     msvcprt:MSVCP110.dll
 0002:0000003c       __imp_?_Xout_of_range@std@@YAXPBD@Z 1000903c     msvcprt:MSVCP110.dll
 0002:00000040       \177MSVCP110_NULL_THUNK_DATA 10009040     msvcprt:MSVCP110.dll
 0002:00000044       __imp__memcpy              10009044     MSVCRT:MSVCR110.dll
 0002:00000048       __imp__strlen              10009048     MSVCRT:MSVCR110.dll
 0002:0000004c       __imp__memmove             1000904c     MSVCRT:MSVCR110.dll
 0002:00000050       __imp___CxxThrowException@8 10009050     MSVCRT:MSVCR110.dll
 0002:00000054       __imp____CxxFrameHandler3  10009054     MSVCRT:MSVCR110.dll
 0002:00000058       __imp__memset              10009058     MSVCRT:MSVCR110.dll
 0002:0000005c       __imp__fclose              1000905c     MSVCRT:MSVCR110.dll
 0002:00000060       __imp___fdopen             10009060     MSVCRT:MSVCR110.dll
 0002:00000064       __imp__ferror              10009064     MSVCRT:MSVCR110.dll
 0002:00000068       __imp__fflush              10009068     MSVCRT:MSVCR110.dll
 0002:0000006c       __imp__fopen               1000906c     MSVCRT:MSVCR110.dll
 0002:00000070       __imp__fprintf             10009070     MSVCRT:MSVCR110.dll
 0002:00000074       __imp__fputc               10009074     MSVCRT:MSVCR110.dll
 0002:00000078       __imp__fread               10009078     MSVCRT:MSVCR110.dll
 0002:0000007c       __imp__fseek               1000907c     MSVCRT:MSVCR110.dll
 0002:00000080       __imp__ftell               10009080     MSVCRT:MSVCR110.dll
 0002:00000084       __imp__fwrite              10009084     MSVCRT:MSVCR110.dll
 0002:00000088       __imp_??3@YAXPAX@Z         10009088     MSVCRT:MSVCR110.dll
 0002:0000008c       __imp__sprintf             1000908c     MSVCRT:MSVCR110.dll
 0002:00000090       __imp__vsprintf            10009090     MSVCRT:MSVCR110.dll
 0002:00000094       __imp_??2@YAPAXI@Z         10009094     MSVCRT:MSVCR110.dll
 0002:00000098       __imp__strcat              10009098     MSVCRT:MSVCR110.dll
 0002:0000009c       __imp___errno              1000909c     MSVCRT:MSVCR110.dll
 0002:000000a0       __imp__free                100090a0     MSVCRT:MSVCR110.dll
 0002:000000a4       __imp__malloc              100090a4     MSVCRT:MSVCR110.dll
 0002:000000a8       __imp__calloc              100090a8     MSVCRT:MSVCR110.dll
 0002:000000ac       __imp___lock               100090ac     MSVCRT:MSVCR110.dll
 0002:000000b0       __imp___unlock             100090b0     MSVCRT:MSVCR110.dll
 0002:000000b4       __imp___calloc_crt         100090b4     MSVCRT:MSVCR110.dll
 0002:000000b8       __imp____dllonexit         100090b8     MSVCRT:MSVCR110.dll
 0002:000000bc       __imp___onexit             100090bc     MSVCRT:MSVCR110.dll
 0002:000000c0       __imp_??1type_info@@UAE@XZ 100090c0     MSVCRT:MSVCR110.dll
 0002:000000c4       __imp____CppXcptFilter     100090c4     MSVCRT:MSVCR110.dll
 0002:000000c8       __imp___amsg_exit          100090c8     MSVCRT:MSVCR110.dll
 0002:000000cc       __imp___malloc_crt         100090cc     MSVCRT:MSVCR110.dll
 0002:000000d0       __imp___initterm           100090d0     MSVCRT:MSVCR110.dll
 0002:000000d4       __imp___initterm_e         100090d4     MSVCRT:MSVCR110.dll
 0002:000000d8       __imp___except_handler4_common 100090d8     MSVCRT:MSVCR110.dll
 0002:000000dc       __imp_?terminate@@YAXXZ    100090dc     MSVCRT:MSVCR110.dll
 0002:000000e0       __imp____clean_type_info_names_internal 100090e0     MSVCRT:MSVCR110.dll
 0002:000000e4       __imp___crt_debugger_hook  100090e4     MSVCRT:MSVCR110.dll
 0002:000000e8       __imp____crtUnhandledException 100090e8     MSVCRT:MSVCR110.dll
 0002:000000ec       __imp____crtTerminateProcess 100090ec     MSVCRT:MSVCR110.dll
 0002:000000f0       __imp___purecall           100090f0     MSVCRT:MSVCR110.dll
 0002:000000f4       __imp__strcpy              100090f4     MSVCRT:MSVCR110.dll
 0002:000000f8       __imp__rewind              100090f8     MSVCRT:MSVCR110.dll
 0002:000000fc       \177MSVCR110_NULL_THUNK_DATA 100090fc     MSVCRT:MSVCR110.dll
 0002:00000100       __imp_?MemPoolAlloc@@YGPAXPAU_HMEMPOOL@@I@Z 10009100     Memory:Memory.dll
 0002:00000104       __imp_?MemPoolDestroy@@YGXPAU_HMEMPOOL@@@Z 10009104     Memory:Memory.dll
 0002:00000108       __imp_?MemPoolCreate@@YGPAU_HMEMPOOL@@PBDI@Z 10009108     Memory:Memory.dll
 0002:0000010c       __imp_?MemPoolFree@@YGXPAU_HMEMPOOL@@PAX@Z 1000910c     Memory:Memory.dll
 0002:00000110       \177Memory_NULL_THUNK_DATA 10009110     Memory:Memory.dll
 0002:00000114       ___xc_a                    10009114     MSVCRT:cinitexe.obj
 0002:0000012c       ___xc_z                    1000912c     MSVCRT:cinitexe.obj
 0002:00000130       ___xi_a                    10009130     MSVCRT:cinitexe.obj
 0002:0000013c       ___xi_z                    1000913c     MSVCRT:cinitexe.obj
 0002:00000178       ?is_signed@?$numeric_limits@E@std@@2_NB 10009178     ZLibInit.obj
 0002:0000017c       ?digits@?$numeric_limits@E@std@@2HB 1000917c     ZLibInit.obj
 0002:00000180       ?digits10@?$numeric_limits@E@std@@2HB 10009180     ZLibInit.obj
 0002:00000184       ?is_signed@?$numeric_limits@F@std@@2_NB 10009184     ZLibInit.obj
 0002:00000188       ?digits@?$numeric_limits@F@std@@2HB 10009188     ZLibInit.obj
 0002:0000018c       ?digits10@?$numeric_limits@F@std@@2HB 1000918c     ZLibInit.obj
 0002:00000190       ?value@?$integral_constant@I$0A@@std@@2IB 10009190     ZLibInit.obj
 0002:00000194       ?is_signed@?$numeric_limits@G@std@@2_NB 10009194     ZLibInit.obj
 0002:00000198       ?digits@?$numeric_limits@G@std@@2HB 10009198     ZLibInit.obj
 0002:0000019c       ?digits10@?$numeric_limits@G@std@@2HB 1000919c     ZLibInit.obj
 0002:000001a0       ?is_signed@?$numeric_limits@H@std@@2_NB 100091a0     ZLibInit.obj
 0002:000001a4       ?digits@?$numeric_limits@H@std@@2HB 100091a4     ZLibInit.obj
 0002:000001a8       ?collate@?$_Locbase@H@std@@2HB 100091a8     ZLibInit.obj
 0002:000001ac       ?ctype@?$_Locbase@H@std@@2HB 100091ac     ZLibInit.obj
 0002:000001b0       ?digits10@?$numeric_limits@H@std@@2HB 100091b0     ZLibInit.obj
 0002:000001b4       ?monetary@?$_Locbase@H@std@@2HB 100091b4     ZLibInit.obj
 0002:000001b8       ?numeric@?$_Locbase@H@std@@2HB 100091b8     ZLibInit.obj
 0002:000001bc       ?time@?$_Locbase@H@std@@2HB 100091bc     ZLibInit.obj
 0002:000001c0       ?messages@?$_Locbase@H@std@@2HB 100091c0     ZLibInit.obj
 0002:000001c4       ?all@?$_Locbase@H@std@@2HB 100091c4     ZLibInit.obj
 0002:000001c8       ?none@?$_Locbase@H@std@@2HB 100091c8     ZLibInit.obj
 0002:000001cc       ?is_signed@?$numeric_limits@I@std@@2_NB 100091cc     ZLibInit.obj
 0002:000001d0       ?digits@?$numeric_limits@I@std@@2HB 100091d0     ZLibInit.obj
 0002:000001d4       ?digits10@?$numeric_limits@I@std@@2HB 100091d4     ZLibInit.obj
 0002:000001d8       ?is_signed@?$numeric_limits@J@std@@2_NB 100091d8     ZLibInit.obj
 0002:000001dc       ?digits@?$numeric_limits@J@std@@2HB 100091dc     ZLibInit.obj
 0002:000001e0       ?digits10@?$numeric_limits@J@std@@2HB 100091e0     ZLibInit.obj
 0002:000001e4       ?value@?$_Sizeof@U_Nil@std@@U12@U12@U12@U12@U12@U12@U12@@std@@2IB 100091e4     ZLibInit.obj
 0002:000001e8       ?is_signed@?$numeric_limits@K@std@@2_NB 100091e8     ZLibInit.obj
 0002:000001ec       ?digits@?$numeric_limits@K@std@@2HB 100091ec     ZLibInit.obj
 0002:000001f0       ?digits10@?$numeric_limits@K@std@@2HB 100091f0     ZLibInit.obj
 0002:000001f4       ?is_signed@?$numeric_limits@_J@std@@2_NB 100091f4     ZLibInit.obj
 0002:000001f8       ?digits@?$numeric_limits@_J@std@@2HB 100091f8     ZLibInit.obj
 0002:000001fc       ?digits10@?$numeric_limits@_J@std@@2HB 100091fc     ZLibInit.obj
 0002:00000200       ?is_signed@?$numeric_limits@_K@std@@2_NB 10009200     ZLibInit.obj
 0002:00000204       ?digits@?$numeric_limits@_K@std@@2HB 10009204     ZLibInit.obj
 0002:00000208       ?digits10@?$numeric_limits@_K@std@@2HB 10009208     ZLibInit.obj
 0002:0000020c       ?value@?$integral_constant@_N$0A@@std@@2_NB 1000920c     ZLibInit.obj
 0002:00000210       ?digits@?$numeric_limits@M@std@@2HB 10009210     ZLibInit.obj
 0002:00000214       ?value@?$integral_constant@_N$00@std@@2_NB 10009214     ZLibInit.obj
 0002:00000218       ?digits10@?$numeric_limits@M@std@@2HB 10009218     ZLibInit.obj
 0002:0000021c       ?max_digits10@?$numeric_limits@M@std@@2HB 1000921c     ZLibInit.obj
 0002:00000220       ?max_exponent@?$numeric_limits@M@std@@2HB 10009220     ZLibInit.obj
 0002:00000224       ?max_exponent10@?$numeric_limits@M@std@@2HB 10009224     ZLibInit.obj
 0002:00000228       ?min_exponent@?$numeric_limits@M@std@@2HB 10009228     ZLibInit.obj
 0002:0000022c       ?min_exponent10@?$numeric_limits@M@std@@2HB 1000922c     ZLibInit.obj
 0002:00000230       ?digits@?$numeric_limits@N@std@@2HB 10009230     ZLibInit.obj
 0002:00000234       ?digits10@?$numeric_limits@N@std@@2HB 10009234     ZLibInit.obj
 0002:00000238       ?max_digits10@?$numeric_limits@N@std@@2HB 10009238     ZLibInit.obj
 0002:0000023c       ?max_exponent@?$numeric_limits@N@std@@2HB 1000923c     ZLibInit.obj
 0002:00000240       ?max_exponent10@?$numeric_limits@N@std@@2HB 10009240     ZLibInit.obj
 0002:00000244       ?min_exponent@?$numeric_limits@N@std@@2HB 10009244     ZLibInit.obj
 0002:00000248       ?min_exponent10@?$numeric_limits@N@std@@2HB 10009248     ZLibInit.obj
 0002:0000024c       ?digits@?$numeric_limits@O@std@@2HB 1000924c     ZLibInit.obj
 0002:00000250       ?digits10@?$numeric_limits@O@std@@2HB 10009250     ZLibInit.obj
 0002:00000254       ?max_digits10@?$numeric_limits@O@std@@2HB 10009254     ZLibInit.obj
 0002:00000258       ?max_exponent@?$numeric_limits@O@std@@2HB 10009258     ZLibInit.obj
 0002:0000025c       ?max_exponent10@?$numeric_limits@O@std@@2HB 1000925c     ZLibInit.obj
 0002:00000260       ?min_exponent@?$numeric_limits@O@std@@2HB 10009260     ZLibInit.obj
 0002:00000264       ?min_exponent10@?$numeric_limits@O@std@@2HB 10009264     ZLibInit.obj
 0002:00000268       ?has_denorm@_Num_base@std@@2W4float_denorm_style@2@B 10009268     ZLibInit.obj
 0002:0000026c       ?has_denorm_loss@_Num_base@std@@2_NB 1000926c     ZLibInit.obj
 0002:0000026d       ?has_infinity@_Num_base@std@@2_NB 1000926d     ZLibInit.obj
 0002:0000026e       ?has_quiet_NaN@_Num_base@std@@2_NB 1000926e     ZLibInit.obj
 0002:0000026f       ?has_signaling_NaN@_Num_base@std@@2_NB 1000926f     ZLibInit.obj
 0002:00000270       ?is_bounded@_Num_base@std@@2_NB 10009270     ZLibInit.obj
 0002:00000271       ?is_exact@_Num_base@std@@2_NB 10009271     ZLibInit.obj
 0002:00000272       ?is_iec559@_Num_base@std@@2_NB 10009272     ZLibInit.obj
 0002:00000273       ?is_integer@_Num_base@std@@2_NB 10009273     ZLibInit.obj
 0002:00000274       ?is_modulo@_Num_base@std@@2_NB 10009274     ZLibInit.obj
 0002:00000275       ?is_signed@_Num_base@std@@2_NB 10009275     ZLibInit.obj
 0002:00000276       ?is_specialized@_Num_base@std@@2_NB 10009276     ZLibInit.obj
 0002:00000277       ?tinyness_before@_Num_base@std@@2_NB 10009277     ZLibInit.obj
 0002:00000278       ?traps@_Num_base@std@@2_NB 10009278     ZLibInit.obj
 0002:0000027c       ?round_style@_Num_base@std@@2W4float_round_style@2@B 1000927c     ZLibInit.obj
 0002:00000280       ?digits@_Num_base@std@@2HB 10009280     ZLibInit.obj
 0002:00000284       ?digits10@_Num_base@std@@2HB 10009284     ZLibInit.obj
 0002:00000288       ?max_digits10@_Num_base@std@@2HB 10009288     ZLibInit.obj
 0002:0000028c       ?max_exponent@_Num_base@std@@2HB 1000928c     ZLibInit.obj
 0002:00000290       ?max_exponent10@_Num_base@std@@2HB 10009290     ZLibInit.obj
 0002:00000294       ?min_exponent@_Num_base@std@@2HB 10009294     ZLibInit.obj
 0002:00000298       ?min_exponent10@_Num_base@std@@2HB 10009298     ZLibInit.obj
 0002:0000029c       ?radix@_Num_base@std@@2HB  1000929c     ZLibInit.obj
 0002:000002a0       ?is_bounded@_Num_int_base@std@@2_NB 100092a0     ZLibInit.obj
 0002:000002a1       ?is_exact@_Num_int_base@std@@2_NB 100092a1     ZLibInit.obj
 0002:000002a2       ?is_integer@_Num_int_base@std@@2_NB 100092a2     ZLibInit.obj
 0002:000002a3       ?is_modulo@_Num_int_base@std@@2_NB 100092a3     ZLibInit.obj
 0002:000002a4       ?is_specialized@_Num_int_base@std@@2_NB 100092a4     ZLibInit.obj
 0002:000002a8       ?radix@_Num_int_base@std@@2HB 100092a8     ZLibInit.obj
 0002:000002ac       ?value@?$_Sizeof@HU_Nil@std@@U12@U12@U12@U12@U12@U12@@std@@2IB 100092ac     ZLibInit.obj
 0002:000002b0       ?has_denorm@_Num_float_base@std@@2W4float_denorm_style@2@B 100092b0     ZLibInit.obj
 0002:000002b4       ?has_denorm_loss@_Num_float_base@std@@2_NB 100092b4     ZLibInit.obj
 0002:000002b5       ?has_infinity@_Num_float_base@std@@2_NB 100092b5     ZLibInit.obj
 0002:000002b6       ?has_quiet_NaN@_Num_float_base@std@@2_NB 100092b6     ZLibInit.obj
 0002:000002b7       ?has_signaling_NaN@_Num_float_base@std@@2_NB 100092b7     ZLibInit.obj
 0002:000002b8       ?skipws@?$_Iosb@H@std@@2W4_Fmtflags@12@B 100092b8     ZLibInit.obj
 0002:000002bc       ?unitbuf@?$_Iosb@H@std@@2W4_Fmtflags@12@B 100092bc     ZLibInit.obj
 0002:000002c0       ?is_bounded@_Num_float_base@std@@2_NB 100092c0     ZLibInit.obj
 0002:000002c1       ?is_exact@_Num_float_base@std@@2_NB 100092c1     ZLibInit.obj
 0002:000002c4       ?uppercase@?$_Iosb@H@std@@2W4_Fmtflags@12@B 100092c4     ZLibInit.obj
 0002:000002c8       ?is_iec559@_Num_float_base@std@@2_NB 100092c8     ZLibInit.obj
 0002:000002cc       ?showbase@?$_Iosb@H@std@@2W4_Fmtflags@12@B 100092cc     ZLibInit.obj
 0002:000002d0       ?showpoint@?$_Iosb@H@std@@2W4_Fmtflags@12@B 100092d0     ZLibInit.obj
 0002:000002d4       ?is_integer@_Num_float_base@std@@2_NB 100092d4     ZLibInit.obj
 0002:000002d5       ?is_modulo@_Num_float_base@std@@2_NB 100092d5     ZLibInit.obj
 0002:000002d8       ?showpos@?$_Iosb@H@std@@2W4_Fmtflags@12@B 100092d8     ZLibInit.obj
 0002:000002dc       ?is_signed@_Num_float_base@std@@2_NB 100092dc     ZLibInit.obj
 0002:000002e0       ?left@?$_Iosb@H@std@@2W4_Fmtflags@12@B 100092e0     ZLibInit.obj
 0002:000002e4       ?right@?$_Iosb@H@std@@2W4_Fmtflags@12@B 100092e4     ZLibInit.obj
 0002:000002e8       ?is_specialized@_Num_float_base@std@@2_NB 100092e8     ZLibInit.obj
 0002:000002ec       ?internal@?$_Iosb@H@std@@2W4_Fmtflags@12@B 100092ec     ZLibInit.obj
 0002:000002f0       ?tinyness_before@_Num_float_base@std@@2_NB 100092f0     ZLibInit.obj
 0002:000002f4       ?dec@?$_Iosb@H@std@@2W4_Fmtflags@12@B 100092f4     ZLibInit.obj
 0002:000002f8       ?traps@_Num_float_base@std@@2_NB 100092f8     ZLibInit.obj
 0002:000002fc       ?round_style@_Num_float_base@std@@2W4float_round_style@2@B 100092fc     ZLibInit.obj
 0002:00000300       ?oct@?$_Iosb@H@std@@2W4_Fmtflags@12@B 10009300     ZLibInit.obj
 0002:00000304       ?hex@?$_Iosb@H@std@@2W4_Fmtflags@12@B 10009304     ZLibInit.obj
 0002:00000308       ?radix@_Num_float_base@std@@2HB 10009308     ZLibInit.obj
 0002:0000030c       ?scientific@?$_Iosb@H@std@@2W4_Fmtflags@12@B 1000930c     ZLibInit.obj
 0002:00000310       ?fixed@?$_Iosb@H@std@@2W4_Fmtflags@12@B 10009310     ZLibInit.obj
 0002:00000314       ?hexfloat@?$_Iosb@H@std@@2W4_Fmtflags@12@B 10009314     ZLibInit.obj
 0002:00000318       ?boolalpha@?$_Iosb@H@std@@2W4_Fmtflags@12@B 10009318     ZLibInit.obj
 0002:0000031c       ?_Stdio@?$_Iosb@H@std@@2W4_Fmtflags@12@B 1000931c     ZLibInit.obj
 0002:00000320       ?adjustfield@?$_Iosb@H@std@@2W4_Fmtflags@12@B 10009320     ZLibInit.obj
 0002:00000324       ?is_signed@?$numeric_limits@D@std@@2_NB 10009324     ZLibInit.obj
 0002:00000328       ?basefield@?$_Iosb@H@std@@2W4_Fmtflags@12@B 10009328     ZLibInit.obj
 0002:0000032c       ?floatfield@?$_Iosb@H@std@@2W4_Fmtflags@12@B 1000932c     ZLibInit.obj
 0002:00000330       ?digits@?$numeric_limits@D@std@@2HB 10009330     ZLibInit.obj
 0002:00000334       ?digits10@?$numeric_limits@D@std@@2HB 10009334     ZLibInit.obj
 0002:00000338       ?goodbit@?$_Iosb@H@std@@2W4_Iostate@12@B 10009338     ZLibInit.obj
 0002:0000033c       ?eofbit@?$_Iosb@H@std@@2W4_Iostate@12@B 1000933c     ZLibInit.obj
 0002:00000340       ?failbit@?$_Iosb@H@std@@2W4_Iostate@12@B 10009340     ZLibInit.obj
 0002:00000344       ?badbit@?$_Iosb@H@std@@2W4_Iostate@12@B 10009344     ZLibInit.obj
 0002:00000348       ?_Hardfail@?$_Iosb@H@std@@2W4_Iostate@12@B 10009348     ZLibInit.obj
 0002:0000034c       ?in@?$_Iosb@H@std@@2W4_Openmode@12@B 1000934c     ZLibInit.obj
 0002:00000350       ?out@?$_Iosb@H@std@@2W4_Openmode@12@B 10009350     ZLibInit.obj
 0002:00000354       ?ate@?$_Iosb@H@std@@2W4_Openmode@12@B 10009354     ZLibInit.obj
 0002:00000358       ?app@?$_Iosb@H@std@@2W4_Openmode@12@B 10009358     ZLibInit.obj
 0002:0000035c       ?is_signed@?$numeric_limits@_W@std@@2_NB 1000935c     ZLibInit.obj
 0002:00000360       ?trunc@?$_Iosb@H@std@@2W4_Openmode@12@B 10009360     ZLibInit.obj
 0002:00000364       ?_Nocreate@?$_Iosb@H@std@@2W4_Openmode@12@B 10009364     ZLibInit.obj
 0002:00000368       ?digits@?$numeric_limits@_W@std@@2HB 10009368     ZLibInit.obj
 0002:0000036c       ?_Noreplace@?$_Iosb@H@std@@2W4_Openmode@12@B 1000936c     ZLibInit.obj
 0002:00000370       ?digits10@?$numeric_limits@_W@std@@2HB 10009370     ZLibInit.obj
 0002:00000374       ?binary@?$_Iosb@H@std@@2W4_Openmode@12@B 10009374     ZLibInit.obj
 0002:00000378       ?beg@?$_Iosb@H@std@@2W4_Seekdir@12@B 10009378     ZLibInit.obj
 0002:0000037c       ?cur@?$_Iosb@H@std@@2W4_Seekdir@12@B 1000937c     ZLibInit.obj
 0002:00000380       ?end@?$_Iosb@H@std@@2W4_Seekdir@12@B 10009380     ZLibInit.obj
 0002:00000384       ?is_modulo@?$numeric_limits@_N@std@@2_NB 10009384     ZLibInit.obj
 0002:00000385       ?is_signed@?$numeric_limits@_N@std@@2_NB 10009385     ZLibInit.obj
 0002:00000388       ?digits@?$numeric_limits@_N@std@@2HB 10009388     ZLibInit.obj
 0002:0000038c       ?digits10@?$numeric_limits@_N@std@@2HB 1000938c     ZLibInit.obj
 0002:00000390       ?_Stream_err@failure@ios_base@std@@0W4io_errc@43@B 10009390     ZLibInit.obj
 0002:00000394       ?is_signed@?$numeric_limits@C@std@@2_NB 10009394     ZLibInit.obj
 0002:00000398       ?digits@?$numeric_limits@C@std@@2HB 10009398     ZLibInit.obj
 0002:0000039c       ?digits10@?$numeric_limits@C@std@@2HB 1000939c     ZLibInit.obj
 0002:000003a4       ??_7error_category@std@@6B@ 100093a4     ZLibInit.obj
 0002:000003c0       ??_7_Generic_error_category@std@@6B@ 100093c0     ZLibInit.obj
 0002:000003d8       ??_C@_07DCLBNMLN@generic?$AA@ 100093d8     ZLibInit.obj
 0002:000003e0       ??_C@_0O@BFJCFAAK@unknown?5error?$AA@ 100093e0     ZLibInit.obj
 0002:000003f4       ??_7_Iostream_error_category@std@@6B@ 100093f4     ZLibInit.obj
 0002:0000040c       ??_C@_08LLGCOLLL@iostream?$AA@ 1000940c     ZLibInit.obj
 0002:00000418       ??_C@_0BG@PADBLCHM@iostream?5stream?5error?$AA@ 10009418     ZLibInit.obj
 0002:00000434       ??_7_System_error_category@std@@6B@ 10009434     ZLibInit.obj
 0002:0000044c       ??_C@_06FHFOAHML@system?$AA@ 1000944c     ZLibInit.obj
 0002:00000454       ??_C@_0BI@CFPLBAOH@invalid?5string?5position?$AA@ 10009454     ZLibInit.obj
 0002:0000046c       ??_C@_0BA@JFNIOLAK@string?5too?5long?$AA@ 1000946c     ZLibInit.obj
 0002:0000047c       ??_C@_05HBMFIKCP@1?41?43?$AA@ 1000947c     compress.obj
 0002:00000888       _deflate_copyright         10009888     deflate.obj
 0002:00000938       ??_C@_0BF@FJABJDFD@?$CFc?$CFc?$CFc?$CFc?$CFc?$CFc?$CFc?$CFc?$CFc?$CFc?$AA@ 10009938     gzio.obj
 0002:00000950       ??_C@_07EBNKNFJN@?$DMfd?3?$CFd?$DO?$AA@ 10009950     gzio.obj
 0002:00000958       ??_C@_00CNPNBAHC@?$AA@     10009958     gzio.obj
 0002:0000095c       ??_C@_02LMMGGCAJ@?3?5?$AA@ 1000995c     gzio.obj
 0002:000009ac       ??_C@_0BD@PJCBIDD@invalid?5block?5type?$AA@ 100099ac     infblock.obj
 0002:000009c0       ??_C@_0BN@LGAADGOK@invalid?5stored?5block?5lengths?$AA@ 100099c0     infblock.obj
 0002:000009e0       ??_C@_0CE@GMIGFPBB@too?5many?5length?5or?5distance?5symb@ 100099e0     infblock.obj
 0002:00000a04       ??_C@_0BK@BMMPFBBH@invalid?5bit?5length?5repeat?$AA@ 10009a04     infblock.obj
 0002:00000a20       ??_C@_0BM@FFFLPBBC@invalid?5literal?1length?5code?$AA@ 10009a20     infcodes.obj
 0002:00000a3c       ??_C@_0BG@LBKINIKP@invalid?5distance?5code?$AA@ 10009a3c     infcodes.obj
 0002:00000a58       ??_C@_0BL@IHKGDAEE@unknown?5compression?5method?$AA@ 10009a58     inflate.obj
 0002:00000a74       ??_C@_0BE@EMOGCLGO@invalid?5window?5size?$AA@ 10009a74     inflate.obj
 0002:00000a88       ??_C@_0BH@LIBMMIGA@incorrect?5header?5check?$AA@ 10009a88     inflate.obj
 0002:00000aa0       ??_C@_0BA@MOKMMFOD@need?5dictionary?$AA@ 10009aa0     inflate.obj
 0002:00000ab0       ??_C@_0BF@MEIGEHBE@incorrect?5data?5check?$AA@ 10009ab0     inflate.obj
 0002:00000ac8       _inflate_copyright         10009ac8     inftrees.obj
 0002:00000ce8       ??_C@_0CI@CGMOPDPD@oversubscribed?5dynamic?5bit?5lengt@ 10009ce8     inftrees.obj
 0002:00000d10       ??_C@_0CE@LOHAHEGK@incomplete?5dynamic?5bit?5lengths?5t@ 10009d10     inftrees.obj
 0002:00000d34       ??_C@_0CD@GJIDGCKE@oversubscribed?5literal?1length?5tr@ 10009d34     inftrees.obj
 0002:00000d58       ??_C@_0BP@NEEEJJNA@incomplete?5literal?1length?5tree?$AA@ 10009d58     inftrees.obj
 0002:00000d78       ??_C@_0BN@KBLCDIAI@oversubscribed?5distance?5tree?$AA@ 10009d78     inftrees.obj
 0002:00000d98       ??_C@_0BJ@CBCPDPJF@incomplete?5distance?5tree?$AA@ 10009d98     inftrees.obj
 0002:00000db4       ??_C@_0CB@KPKKKLFO@empty?5distance?5tree?5with?5lengths@ 10009db4     inftrees.obj
 0002:00000dd8       __length_code              10009dd8     trees.obj
 0002:00000ed8       __dist_code                10009ed8     trees.obj
 0002:00001810       ??_C@_0L@FNAOCBOG@stream?5end?$AA@ 1000a810     zutil.obj
 0002:0000181c       ??_C@_0L@KIJFAKBJ@file?5error?$AA@ 1000a81c     zutil.obj
 0002:00001828       ??_C@_0N@MKKNPMJD@stream?5error?$AA@ 1000a828     zutil.obj
 0002:00001838       ??_C@_0L@HAHMBNLP@data?5error?$AA@ 1000a838     zutil.obj
 0002:00001844       ??_C@_0BE@OGGJBMCE@insufficient?5memory?$AA@ 1000a844     zutil.obj
 0002:00001858       ??_C@_0N@DFPGLBGC@buffer?5error?$AA@ 1000a858     zutil.obj
 0002:00001868       ??_C@_0BF@CJFPCCEG@incompatible?5version?$AA@ 1000a868     zutil.obj
 0002:00001880       ??_C@_04IKHBMBIH@ZLib?$AA@ 1000a880     CompressionMem1.obj
 0002:0000188c       ??_7type_info@@6B@         1000a88c     MSVCRT:ti_inst.obj
 0002:00001890       __pDefaultRawDllMain       1000a890     MSVCRT:crtdll.obj
 0002:00001890       __pRawDllMain              1000a890     MSVCRT:crtdll.obj
 0002:00001894       ?ProcessDetach@NativeDll@<CrtImplementationDetails>@@0IB 1000a894     MSVCRT:initsect.obj
 0002:00001898       ?ProcessAttach@NativeDll@<CrtImplementationDetails>@@0IB 1000a898     MSVCRT:initsect.obj
 0002:0000189c       ?ThreadAttach@NativeDll@<CrtImplementationDetails>@@0IB 1000a89c     MSVCRT:initsect.obj
 0002:000018a0       ?ThreadDetach@NativeDll@<CrtImplementationDetails>@@0IB 1000a8a0     MSVCRT:initsect.obj
 0002:000018a4       ?ProcessVerifier@NativeDll@<CrtImplementationDetails>@@0IB 1000a8a4     MSVCRT:initsect.obj
 0002:000018b0       __load_config_used         1000a8b0     MSVCRT:loadcfg.obj
 0002:00001960       ??_R4error_category@std@@6B@ 1000a960     ZLibInit.obj
 0002:00001974       ??_R3error_category@std@@8 1000a974     ZLibInit.obj
 0002:00001984       ??_R2error_category@std@@8 1000a984     ZLibInit.obj
 0002:0000198c       ??_R1A@?0A@EA@error_category@std@@8 1000a98c     ZLibInit.obj
 0002:000019a8       ??_R4_Generic_error_category@std@@6B@ 1000a9a8     ZLibInit.obj
 0002:000019bc       ??_R3_Generic_error_category@std@@8 1000a9bc     ZLibInit.obj
 0002:000019cc       ??_R2_Generic_error_category@std@@8 1000a9cc     ZLibInit.obj
 0002:000019d8       ??_R1A@?0A@EA@_Generic_error_category@std@@8 1000a9d8     ZLibInit.obj
 0002:000019f4       ??_R4_Iostream_error_category@std@@6B@ 1000a9f4     ZLibInit.obj
 0002:00001a08       ??_R3_Iostream_error_category@std@@8 1000aa08     ZLibInit.obj
 0002:00001a18       ??_R2_Iostream_error_category@std@@8 1000aa18     ZLibInit.obj
 0002:00001a28       ??_R1A@?0A@EA@_Iostream_error_category@std@@8 1000aa28     ZLibInit.obj
 0002:00001a44       ??_R4_System_error_category@std@@6B@ 1000aa44     ZLibInit.obj
 0002:00001a58       ??_R3_System_error_category@std@@8 1000aa58     ZLibInit.obj
 0002:00001a68       ??_R2_System_error_category@std@@8 1000aa68     ZLibInit.obj
 0002:00001a78       ??_R1A@?0A@EA@_System_error_category@std@@8 1000aa78     ZLibInit.obj
 0002:00001a94       ??_R4type_info@@6B@        1000aa94     MSVCRT:ti_inst.obj
 0002:00001aa8       ??_R3type_info@@8          1000aaa8     MSVCRT:ti_inst.obj
 0002:00001ab8       ??_R2type_info@@8          1000aab8     MSVCRT:ti_inst.obj
 0002:00001ac0       ??_R1A@?0A@EA@type_info@@8 1000aac0     MSVCRT:ti_inst.obj
 0002:00001ae0       ___safe_se_handler_table   1000aae0     <linker-defined>
 0002:00001ae8       ___rtc_iaa                 1000aae8     MSVCRT:initsect.obj
 0002:00001aec       ___rtc_izz                 1000aaec     MSVCRT:initsect.obj
 0002:00001af0       ___rtc_taa                 1000aaf0     MSVCRT:initsect.obj
 0002:00001af4       ___rtc_tzz                 1000aaf4     MSVCRT:initsect.obj
 0002:00001c2c       __IMPORT_DESCRIPTOR_KERNEL32 1000ac2c     kernel32:KERNEL32.dll
 0002:00001c40       __IMPORT_DESCRIPTOR_Memory 1000ac40     Memory:Memory.dll
 0002:00001c54       __IMPORT_DESCRIPTOR_MSVCP110 1000ac54     msvcprt:MSVCP110.dll
 0002:00001c68       __IMPORT_DESCRIPTOR_MSVCR110 1000ac68     MSVCRT:MSVCR110.dll
 0002:00001c7c       __NULL_IMPORT_DESCRIPTOR   1000ac7c     kernel32:KERNEL32.dll
 0003:00000000       ?_Generic_object@?$_Error_objects@H@std@@2V_Generic_error_category@2@A 1000c000     ZLibInit.obj
 0003:00000004       ?_Iostream_object@?$_Error_objects@H@std@@2V_Iostream_error_category@2@A 1000c004     ZLibInit.obj
 0003:00000008       ?_System_object@?$_Error_objects@H@std@@2V_System_error_category@2@A 1000c008     ZLibInit.obj
 0003:0000000c       ??_R0?AVerror_category@std@@@8 1000c00c     ZLibInit.obj
 0003:00000030       ??_R0?AV_Generic_error_category@std@@@8 1000c030     ZLibInit.obj
 0003:0000005c       ??_R0?AV_Iostream_error_category@std@@@8 1000c05c     ZLibInit.obj
 0003:00000088       ??_R0?AV_System_error_category@std@@@8 1000c088     ZLibInit.obj
 0003:000011c8       _inflate_mask              1000d1c8     infutil.obj
 0003:00001248       _z_errmsg                  1000d248     zutil.obj
 0003:00001270       ??_R0?AVtype_info@@@8      1000d270     MSVCRT:ti_inst.obj
 0003:00001290       ___native_dllmain_reason   1000d290     MSVCRT:natstart.obj
 0003:00001294       ___security_cookie         1000d294     MSVCRT:gs_cookie.obj
 0003:00001298       ___security_cookie_complement 1000d298     MSVCRT:gs_cookie.obj
 0003:000012a4       ?id@?$num_put@DV?$back_insert_iterator@V?$basic_string@DU?$char_traits@D@std@@V?$allocator@D@2@@std@@@std@@@std@@2V0locale@2@A 1000d2a4     ZLibInit.obj
 0003:000012a8       ?id@?$num_put@_WV?$back_insert_iterator@V?$basic_string@_WU?$char_traits@_W@std@@V?$allocator@_W@2@@std@@@std@@@std@@2V0locale@2@A 1000d2a8     ZLibInit.obj
 0003:000012bc       ?__type_info_root_node@@3U__type_info_node@@A 1000d2bc     MSVCRT:tncleanup.obj
 0003:000015e8       ___native_startup_lock     1000d5e8     <common>
 0003:000015ec       ___native_startup_state    1000d5ec     <common>
 0003:000015f0       ___dyn_tls_init_callback   1000d5f0     <common>
 0003:000015f4       ___onexitend               1000d5f4     <common>
 0003:000015f8       ___onexitbegin             1000d5f8     <common>

 entry point at        0001:00006a9a

 Static symbols

 0000:ffff0000       .debug$S                   10000000     MSVCRT:MSVCR110.dll
 0000:ffff0000       .debug$S                   10000000     MSVCRT:MSVCR110.dll
 0000:ffff0000       .debug$S                   10000000     MSVCRT:MSVCR110.dll
 0000:ffff0000       .debug$S                   10000000     MSVCRT:MSVCR110.dll
 0000:ffff0000       .debug$S                   10000000     MSVCRT:MSVCR110.dll
 0000:ffff0000       .debug$S                   10000000     MSVCRT:MSVCR110.dll
 0000:ffff0000       .debug$S                   10000000     MSVCRT:MSVCR110.dll
 0000:ffff0000       .debug$S                   10000000     MSVCRT:MSVCR110.dll
 0000:ffff0000       .debug$S                   10000000     MSVCRT:MSVCR110.dll
 0000:ffff0000       .debug$S                   10000000     MSVCRT:MSVCR110.dll
 0000:ffff0000       .debug$S                   10000000     MSVCRT:MSVCR110.dll
 0000:ffff0000       .debug$S                   10000000     MSVCRT:MSVCR110.dll
 0000:ffff0000       .debug$S                   10000000     MSVCRT:MSVCR110.dll
 0000:ffff0000       .debug$S                   10000000     MSVCRT:MSVCR110.dll
 0000:ffff0000       .debug$S                   10000000     MSVCRT:MSVCR110.dll
 0000:ffff0000       .debug$S                   10000000     MSVCRT:MSVCR110.dll
 0000:ffff0000       .debug$S                   10000000     MSVCRT:MSVCR110.dll
 0000:ffff0000       .debug$S                   10000000     MSVCRT:MSVCR110.dll
 0000:ffff0000       .debug$S                   10000000     MSVCRT:MSVCR110.dll
 0000:ffff0000       .debug$S                   10000000     MSVCRT:MSVCR110.dll
 0000:ffff0000       .debug$S                   10000000     MSVCRT:MSVCR110.dll
 0000:ffff0000       .debug$S                   10000000     MSVCRT:MSVCR110.dll
 0000:ffff0000       .debug$S                   10000000     MSVCRT:MSVCR110.dll
 0000:ffff0000       .debug$S                   10000000     MSVCRT:MSVCR110.dll
 0000:ffff0000       .debug$S                   10000000     MSVCRT:MSVCR110.dll
 0000:ffff0000       .debug$S                   10000000     MSVCRT:MSVCR110.dll
 0000:ffff0000       .debug$S                   10000000     MSVCRT:MSVCR110.dll
 0000:ffff0000       .debug$S                   10000000     MSVCRT:MSVCR110.dll
 0000:ffff0000       .debug$S                   10000000     MSVCRT:MSVCR110.dll
 0000:ffff0000       .debug$S                   10000000     MSVCRT:MSVCR110.dll
 0000:ffff0000       .debug$S                   10000000     MSVCRT:MSVCR110.dll
 0000:ffff0000       .debug$S                   10000000     MSVCRT:MSVCR110.dll
 0000:ffff0000       .debug$S                   10000000     MSVCRT:MSVCR110.dll
 0000:ffff0000       .debug$S                   10000000     MSVCRT:MSVCR110.dll
 0000:ffff0000       .debug$S                   10000000     MSVCRT:MSVCR110.dll
 0000:ffff0000       .debug$S                   10000000     MSVCRT:MSVCR110.dll
 0000:ffff0000       .debug$S                   10000000     MSVCRT:MSVCR110.dll
 0000:ffff0000       .debug$S                   10000000     MSVCRT:MSVCR110.dll
 0000:ffff0000       .debug$S                   10000000     MSVCRT:MSVCR110.dll
 0000:ffff0000       .debug$S                   10000000     MSVCRT:MSVCR110.dll
 0000:ffff0000       .debug$S                   10000000     MSVCRT:MSVCR110.dll
 0000:ffff0000       .debug$S                   10000000     MSVCRT:MSVCR110.dll
 0000:ffff0000       .debug$S                   10000000     MSVCRT:MSVCR110.dll
 0000:ffff0000       .debug$S                   10000000     MSVCRT:MSVCR110.dll
 0000:ffff0000       .debug$S                   10000000     MSVCRT:MSVCR110.dll
 0000:ffff0000       .debug$S                   10000000     MSVCRT:MSVCR110.dll
 0000:ffff0000       .debug$S                   10000000     msvcprt:MSVCP110.dll
 0000:ffff0000       .debug$S                   10000000     msvcprt:MSVCP110.dll
 0000:ffff0000       .debug$S                   10000000     msvcprt:MSVCP110.dll
 0000:ffff0000       .debug$S                   10000000     msvcprt:MSVCP110.dll
 0000:ffff0000       .debug$S                   10000000     msvcprt:MSVCP110.dll
 0000:ffff0000       .debug$S                   10000000     Memory:Memory.dll
 0000:ffff0000       .debug$S                   10000000     Memory:Memory.dll
 0000:ffff0000       .debug$S                   10000000     Memory:Memory.dll
 0000:ffff0000       .debug$S                   10000000     Memory:Memory.dll
 0000:ffff0000       .debug$S                   10000000     kernel32:KERNEL32.dll
 0000:ffff0000       .debug$S                   10000000     kernel32:KERNEL32.dll
 0000:ffff0000       .debug$S                   10000000     kernel32:KERNEL32.dll
 0000:ffff0000       .debug$S                   10000000     kernel32:KERNEL32.dll
 0000:ffff0000       .debug$S                   10000000     kernel32:KERNEL32.dll
 0000:ffff0000       .debug$S                   10000000     kernel32:KERNEL32.dll
 0001:fffff000       __ehhandler$?_Copy@?$basic_string@DU?$char_traits@D@std@@V?$allocator@D@2@@std@@QAEXII@Z 10000000 f   CompressionMem1.obj
 0002:ffff7000       ?id$initializer$@?$num_put@_WV?$back_insert_iterator@V?$basic_string@_WU?$char_traits@_W@std@@V?$allocator@_W@2@@std@@@std@@@std@@2P6AXXZA 10000000     pch.obj
 0002:ffff7000       ?id$initializer$@?$num_put@DV?$back_insert_iterator@V?$basic_string@DU?$char_traits@D@std@@V?$allocator@D@2@@std@@@std@@@std@@2P6AXXZA 10000000     pch.obj
 0002:ffff7000       ?_Iostream_object$initializer$@?$_Error_objects@H@std@@2P6AXXZA 10000000     Compression1.obj
 0002:ffff7000       __catchsym$?_Copy@?$basic_string@DU?$char_traits@D@std@@V?$allocator@D@2@@std@@QAEXII@Z$5 10000000     Compression1.obj
 0002:ffff7000       ?_System_object$initializer$@?$_Error_objects@H@std@@2P6AXXZA 10000000     pch.obj
 0002:ffff7000       ?_System_object$initializer$@?$_Error_objects@H@std@@2P6AXXZA 10000000     Compression1.obj
 0002:ffff7000       __catchsym$?_Copy@?$basic_string@DU?$char_traits@D@std@@V?$allocator@D@2@@std@@QAEXII@Z$5 10000000     CompressionMem1.obj
 0000:ffff0000       .debug$S                   10000000     kernel32:KERNEL32.dll
 0000:ffff0000       .debug$S                   10000000     kernel32:KERNEL32.dll
 0000:ffff0000       .debug$S                   10000000     kernel32:KERNEL32.dll
 0002:ffff7000       ?_Generic_object$initializer$@?$_Error_objects@H@std@@2P6AXXZA 10000000     CompressionMem1.obj
 0002:ffff7000       ?_Iostream_object$initializer$@?$_Error_objects@H@std@@2P6AXXZA 10000000     CompressionMem1.obj
 0002:ffff7000       ?_System_object$initializer$@?$_Error_objects@H@std@@2P6AXXZA 10000000     CompressionMem1.obj
 0002:ffff7000       ?id$initializer$@?$num_put@DV?$back_insert_iterator@V?$basic_string@DU?$char_traits@D@std@@V?$allocator@D@2@@std@@@std@@@std@@2P6AXXZA 10000000     CompressionMem1.obj
 0002:ffff7000       ?id$initializer$@?$num_put@_WV?$back_insert_iterator@V?$basic_string@_WU?$char_traits@_W@std@@V?$allocator@_W@2@@std@@@std@@@std@@2P6AXXZA 10000000     CompressionMem1.obj
 0000:ffff0000       .debug$S                   10000000     kernel32:KERNEL32.dll
 0002:ffff7000       ?_Iostream_object$initializer$@?$_Error_objects@H@std@@2P6AXXZA 10000000     pch.obj
 0002:ffff7000       ?_Generic_object$initializer$@?$_Error_objects@H@std@@2P6AXXZA 10000000     pch.obj
 0002:ffff7000       __catchsym$?_Copy@?$basic_string@DU?$char_traits@D@std@@V?$allocator@D@2@@std@@QAEXII@Z$5 10000000     pch.obj
 0002:ffff7000       ?id$initializer$@?$num_put@DV?$back_insert_iterator@V?$basic_string@DU?$char_traits@D@std@@V?$allocator@D@2@@std@@@std@@@std@@2P6AXXZA 10000000     Compression1.obj
 0002:ffff7000       ?id$initializer$@?$num_put@_WV?$back_insert_iterator@V?$basic_string@_WU?$char_traits@_W@std@@V?$allocator@_W@2@@std@@@std@@@std@@2P6AXXZA 10000000     Compression1.obj
 0001:fffff000       __ehhandler$?_Copy@?$basic_string@DU?$char_traits@D@std@@V?$allocator@D@2@@std@@QAEXII@Z 10000000 f   Compression1.obj
 0001:fffff000       __ehhandler$?_Copy@?$basic_string@DU?$char_traits@D@std@@V?$allocator@D@2@@std@@QAEXII@Z 10000000 f   pch.obj
 0002:ffff7000       ?_Generic_object$initializer$@?$_Error_objects@H@std@@2P6AXXZA 10000000     Compression1.obj
 0002:ffff7010       __catchsym$?_Copy@?$basic_string@DU?$char_traits@D@std@@V?$allocator@D@2@@std@@QAEXII@Z$4 10000010     Compression1.obj
 0002:ffff7010       __catchsym$?_Copy@?$basic_string@DU?$char_traits@D@std@@V?$allocator@D@2@@std@@QAEXII@Z$4 10000010     pch.obj
 0002:ffff7010       __catchsym$?_Copy@?$basic_string@DU?$char_traits@D@std@@V?$allocator@D@2@@std@@QAEXII@Z$4 10000010     CompressionMem1.obj
 0002:ffff7020       __unwindtable$?_Copy@?$basic_string@DU?$char_traits@D@std@@V?$allocator@D@2@@std@@QAEXII@Z 10000020     CompressionMem1.obj
 0002:ffff7020       __unwindtable$?_Copy@?$basic_string@DU?$char_traits@D@std@@V?$allocator@D@2@@std@@QAEXII@Z 10000020     pch.obj
 0002:ffff7020       __unwindtable$?_Copy@?$basic_string@DU?$char_traits@D@std@@V?$allocator@D@2@@std@@QAEXII@Z 10000020     Compression1.obj
 0002:ffff7040       __ehfuncinfo$?_Copy@?$basic_string@DU?$char_traits@D@std@@V?$allocator@D@2@@std@@QAEXII@Z 10000040     CompressionMem1.obj
 0002:ffff7040       __ehfuncinfo$?_Copy@?$basic_string@DU?$char_traits@D@std@@V?$allocator@D@2@@std@@QAEXII@Z 10000040     pch.obj
 0002:ffff7040       __ehfuncinfo$?_Copy@?$basic_string@DU?$char_traits@D@std@@V?$allocator@D@2@@std@@QAEXII@Z 10000040     Compression1.obj
 0002:ffff7064       __tryblocktable$?_Copy@?$basic_string@DU?$char_traits@D@std@@V?$allocator@D@2@@std@@QAEXII@Z 10000064     CompressionMem1.obj
 0002:ffff7064       __tryblocktable$?_Copy@?$basic_string@DU?$char_traits@D@std@@V?$allocator@D@2@@std@@QAEXII@Z 10000064     Compression1.obj
 0002:ffff7064       __tryblocktable$?_Copy@?$basic_string@DU?$char_traits@D@std@@V?$allocator@D@2@@std@@QAEXII@Z 10000064     pch.obj
 0001:fffff068       __catch$?_Copy@?$basic_string@DU?$char_traits@D@std@@V?$allocator@D@2@@std@@QAEXII@Z$0 10000068 f   Compression1.obj
 0001:fffff068       __catch$?_Copy@?$basic_string@DU?$char_traits@D@std@@V?$allocator@D@2@@std@@QAEXII@Z$0 10000068 f   pch.obj
 0001:fffff068       __catch$?_Copy@?$basic_string@DU?$char_traits@D@std@@V?$allocator@D@2@@std@@QAEXII@Z$0 10000068 f   CompressionMem1.obj
 0001:fffff0ee       __catch$?_Copy@?$basic_string@DU?$char_traits@D@std@@V?$allocator@D@2@@std@@QAEXII@Z$1 100000ee f   Compression1.obj
 0001:fffff0ee       __catch$?_Copy@?$basic_string@DU?$char_traits@D@std@@V?$allocator@D@2@@std@@QAEXII@Z$1 100000ee f   CompressionMem1.obj
 0001:fffff0ee       __catch$?_Copy@?$basic_string@DU?$char_traits@D@std@@V?$allocator@D@2@@std@@QAEXII@Z$1 100000ee f   pch.obj
 0001:0000023f       __catch$?_Copy@?$basic_string@DU?$char_traits@D@std@@V?$allocator@D@2@@std@@QAEXII@Z$0 1000123f f i ZLibInit.obj
 0001:000002c5       __catch$?_Copy@?$basic_string@DU?$char_traits@D@std@@V?$allocator@D@2@@std@@QAEXII@Z$1 100012c5 f i ZLibInit.obj
 0001:00000a76       _deflate_stored@8          10001a76 f   deflate.obj
 0001:00000b9b       _deflate_fast@8            10001b9b f   deflate.obj
 0001:00000e53       _deflate_slow@8            10001e53 f   deflate.obj
 0001:000019ec       _fill_window@4             100029ec f   deflate.obj
 0001:00001b4a       _flush_pending@4           10002b4a f   deflate.obj
 0001:00001b99       _lm_init@4                 10002b99 f   deflate.obj
 0001:00001c1e       _longest_match@8           10002c1e f   deflate.obj
 0001:00001d81       _putShortMSB@8             10002d81 f   deflate.obj
 0001:00001dad       _read_buf@12               10002dad f   deflate.obj
 0001:00001e00       _check_header@4            10002e00 f   gzio.obj
 0001:00001eec       _destroy@4                 10002eec f   gzio.obj
 0001:00001f8d       _do_flush@8                10002f8d f   gzio.obj
 0001:00002032       _getLong@4                 10003032 f   gzio.obj
 0001:00002072       _get_byte@4                10003072 f   gzio.obj
 0001:000020de       _gz_open@12                100030de f   gzio.obj
 0001:00002985       _putLong@8                 10003985 f   gzio.obj
 0001:00003221       $LN174                     10004221     infblock.obj
 0001:000039bf       $LN107                     100049bf     infcodes.obj
 0001:00004090       $LN58                      10005090     inflate.obj
 0001:00004364       _huft_build@40             10005364 f   inftrees.obj
 0001:00004f66       _bi_flush@4                10005f66 f   trees.obj
 0001:00004fd4       _bi_reverse@8              10005fd4 f   trees.obj
 0001:00004ff7       _bi_windup@4               10005ff7 f   trees.obj
 0001:00005050       _build_bl_tree@4           10006050 f   trees.obj
 0001:000050b7       _build_tree@8              100060b7 f   trees.obj
 0001:00005301       _compress_block@12         10006301 f   trees.obj
 0001:000056ad       _copy_block@16             100066ad f   trees.obj
 0001:0000572f       _gen_bitlen@8              1000672f f   trees.obj
 0001:00005967       _gen_codes@12              10006967 f   trees.obj
 0001:000059de       _init_block@4              100069de f   trees.obj
 0001:00005a49       _pqdownheap@12             10006a49 f   trees.obj
 0001:00005b0d       _scan_tree@12              10006b0d f   trees.obj
 0001:00005bdb       _send_all_trees@16         10006bdb f   trees.obj
 0001:00005df9       _send_tree@12              10006df9 f   trees.obj
 0001:000062b7       _set_data_type@4           100072b7 f   trees.obj
 0001:00006312       _tr_static_init@0          10007312 f   trees.obj
 0001:00006728       $$000000                   10007728     MSVCRT:ehprolog.obj
 0001:00006820       $$000000                   10007820     MSVCRT:chkstk.obj
 0001:00006852       _pre_c_init                10007852 f   MSVCRT:crtdll.obj
 0001:00006abd       ___DllMainCRTStartup       10007abd f   MSVCRT:crtdll.obj
 0001:00006c10       $$000000                   10007c10     MSVCRT:sehprolg4.obj
 0001:00006cfb       ?ArrayUnwindFilter@@YAHPAU_EXCEPTION_POINTERS@@@Z 10007cfb f   MSVCRT:ehvecdtr.obj
 0001:00007352       __ehhandler$?_Copy@?$basic_string@DU?$char_traits@D@std@@V?$allocator@D@2@@std@@QAEXII@Z 10008352 f   ZLibInit.obj
 0001:0000735c       ??__E?_Generic_object@?$_Error_objects@H@std@@2V_Generic_error_category@2@A@@YAXXZ 1000835c f   ZLibInit.obj
 0001:00007368       ??__E?_Iostream_object@?$_Error_objects@H@std@@2V_Iostream_error_category@2@A@@YAXXZ 10008368 f   ZLibInit.obj
 0001:00007374       ??__E?_System_object@?$_Error_objects@H@std@@2V_System_error_category@2@A@@YAXXZ 10008374 f   ZLibInit.obj
 0001:00007380       ??__E?id@?$num_put@DV?$back_insert_iterator@V?$basic_string@DU?$char_traits@D@std@@V?$allocator@D@2@@std@@@std@@@std@@2V0locale@2@A@@YAXXZ 10008380 f   ZLibInit.obj
 0001:00007388       ??__E?id@?$num_put@_WV?$back_insert_iterator@V?$basic_string@_WU?$char_traits@_W@std@@V?$allocator@_W@2@@std@@@std@@@std@@2V0locale@2@A@@YAXXZ 10008388 f   ZLibInit.obj
 0001:00007390       ??__E?_Generic_object@?$_Error_objects@H@std@@2V_Generic_error_category@2@A@@YAXXZ 10008390 f   pch.obj
 0001:0000739c       ??__E?_Iostream_object@?$_Error_objects@H@std@@2V_Iostream_error_category@2@A@@YAXXZ 1000839c f   pch.obj
 0001:000073a8       ??__E?_System_object@?$_Error_objects@H@std@@2V_System_error_category@2@A@@YAXXZ 100083a8 f   pch.obj
 0001:000073b4       ??__E?id@?$num_put@DV?$back_insert_iterator@V?$basic_string@DU?$char_traits@D@std@@V?$allocator@D@2@@std@@@std@@@std@@2V0locale@2@A@@YAXXZ 100083b4 f   pch.obj
 0001:000073bc       ??__E?id@?$num_put@_WV?$back_insert_iterator@V?$basic_string@_WU?$char_traits@_W@std@@V?$allocator@_W@2@@std@@@std@@@std@@2V0locale@2@A@@YAXXZ 100083bc f   pch.obj
 0001:000073c4       ??__E?_Generic_object@?$_Error_objects@H@std@@2V_Generic_error_category@2@A@@YAXXZ 100083c4 f   Compression1.obj
 0001:000073d0       ??__E?_Iostream_object@?$_Error_objects@H@std@@2V_Iostream_error_category@2@A@@YAXXZ 100083d0 f   Compression1.obj
 0001:000073dc       ??__E?_System_object@?$_Error_objects@H@std@@2V_System_error_category@2@A@@YAXXZ 100083dc f   Compression1.obj
 0001:000073e8       ??__E?id@?$num_put@DV?$back_insert_iterator@V?$basic_string@DU?$char_traits@D@std@@V?$allocator@D@2@@std@@@std@@@std@@2V0locale@2@A@@YAXXZ 100083e8 f   Compression1.obj
 0001:000073f0       ??__E?id@?$num_put@_WV?$back_insert_iterator@V?$basic_string@_WU?$char_traits@_W@std@@V?$allocator@_W@2@@std@@@std@@@std@@2V0locale@2@A@@YAXXZ 100083f0 f   Compression1.obj
 0001:000073f8       ??__E?_Generic_object@?$_Error_objects@H@std@@2V_Generic_error_category@2@A@@YAXXZ 100083f8 f   CompressionMem1.obj
 0001:00007404       ??__E?_Iostream_object@?$_Error_objects@H@std@@2V_Iostream_error_category@2@A@@YAXXZ 10008404 f   CompressionMem1.obj
 0001:00007410       ??__E?_System_object@?$_Error_objects@H@std@@2V_System_error_category@2@A@@YAXXZ 10008410 f   CompressionMem1.obj
 0001:0000741c       ??__E?id@?$num_put@DV?$back_insert_iterator@V?$basic_string@DU?$char_traits@D@std@@V?$allocator@D@2@@std@@@std@@@std@@2V0locale@2@A@@YAXXZ 1000841c f   CompressionMem1.obj
 0001:00007424       ??__E?id@?$num_put@_WV?$back_insert_iterator@V?$basic_string@_WU?$char_traits@_W@std@@V?$allocator@_W@2@@std@@@std@@@std@@2V0locale@2@A@@YAXXZ 10008424 f   CompressionMem1.obj
 0001:0000742c       ??__F?_Generic_object@?$_Error_objects@H@std@@2V_Generic_error_category@2@A@@YAXXZ 1000842c f   ZLibInit.obj
 0001:00007437       ??__F?_Iostream_object@?$_Error_objects@H@std@@2V_Iostream_error_category@2@A@@YAXXZ 10008437 f   ZLibInit.obj
 0001:00007442       ??__F?_System_object@?$_Error_objects@H@std@@2V_System_error_category@2@A@@YAXXZ 10008442 f   ZLibInit.obj
 0001:0000744d       ??__F?_Generic_object@?$_Error_objects@H@std@@2V_Generic_error_category@2@A@@YAXXZ 1000844d f   pch.obj
 0001:00007458       ??__F?_Iostream_object@?$_Error_objects@H@std@@2V_Iostream_error_category@2@A@@YAXXZ 10008458 f   pch.obj
 0001:00007463       ??__F?_System_object@?$_Error_objects@H@std@@2V_System_error_category@2@A@@YAXXZ 10008463 f   pch.obj
 0001:0000746e       ??__F?_Generic_object@?$_Error_objects@H@std@@2V_Generic_error_category@2@A@@YAXXZ 1000846e f   Compression1.obj
 0001:00007479       ??__F?_Iostream_object@?$_Error_objects@H@std@@2V_Iostream_error_category@2@A@@YAXXZ 10008479 f   Compression1.obj
 0001:00007484       ??__F?_System_object@?$_Error_objects@H@std@@2V_System_error_category@2@A@@YAXXZ 10008484 f   Compression1.obj
 0001:0000748f       ??__F?_Generic_object@?$_Error_objects@H@std@@2V_Generic_error_category@2@A@@YAXXZ 1000848f f   CompressionMem1.obj
 0001:0000749a       ??__F?_Iostream_object@?$_Error_objects@H@std@@2V_Iostream_error_category@2@A@@YAXXZ 1000849a f   CompressionMem1.obj
 0001:000074a5       ??__F?_System_object@?$_Error_objects@H@std@@2V_System_error_category@2@A@@YAXXZ 100084a5 f   CompressionMem1.obj
 0002:00000118       ?_Generic_object$initializer$@?$_Error_objects@H@std@@2P6AXXZA 10009118     ZLibInit.obj
 0002:0000011c       ?_Iostream_object$initializer$@?$_Error_objects@H@std@@2P6AXXZA 1000911c     ZLibInit.obj
 0002:00000120       ?_System_object$initializer$@?$_Error_objects@H@std@@2P6AXXZA 10009120     ZLibInit.obj
 0002:00000124       ?id$initializer$@?$num_put@DV?$back_insert_iterator@V?$basic_string@DU?$char_traits@D@std@@V?$allocator@D@2@@std@@@std@@@std@@2P6AXXZA 10009124     ZLibInit.obj
 0002:00000128       ?id$initializer$@?$num_put@_WV?$back_insert_iterator@V?$basic_string@_WU?$char_traits@_W@std@@V?$allocator@_W@2@@std@@@std@@@std@@2P6AXXZA 10009128     ZLibInit.obj
 0002:00000134       _pcinit                    10009134     MSVCRT:crtdll.obj
 0002:00000138       _pinit                     10009138     MSVCRT:atonexit.obj
 0002:00000488       _crc_table                 10009488     crc32.obj
 0002:000008c0       _configuration_table       100098c0     deflate.obj
 0002:00000960       _border                    10009960     infblock.obj
 0002:00000a54       ?mark@?3??inflateSync@@9@9 10009a54     inflate.obj
 0002:00000af8       _cplens                    10009af8     inftrees.obj
 0002:00000b78       _cplext                    10009b78     inftrees.obj
 0002:00000bf8       _cpdist                    10009bf8     inftrees.obj
 0002:00000c70       _cpdext                    10009c70     inftrees.obj
 0002:000010d8       _extra_lbits               1000a0d8     trees.obj
 0002:0000114c       _bl_order                  1000a14c     trees.obj
 0002:00001160       _extra_dbits               1000a160     trees.obj
 0002:000011d8       _extra_blbits              1000a1d8     trees.obj
 0002:00001228       _static_ltree              1000a228     trees.obj
 0002:000016a8       _static_dtree              1000a6a8     trees.obj
 0002:00001720       _base_length               1000a720     trees.obj
 0002:00001798       _base_dist                 1000a798     trees.obj
 0002:000018a8       _GS_ExceptionPointers      1000a8a8     MSVCRT:gs_report.obj
 0002:00001af8       __catchsym$?_Copy@?$basic_string@DU?$char_traits@D@std@@V?$allocator@D@2@@std@@QAEXII@Z$5 1000aaf8     ZLibInit.obj
 0002:00001b08       __catchsym$?_Copy@?$basic_string@DU?$char_traits@D@std@@V?$allocator@D@2@@std@@QAEXII@Z$4 1000ab08     ZLibInit.obj
 0002:00001b18       __unwindtable$?_Copy@?$basic_string@DU?$char_traits@D@std@@V?$allocator@D@2@@std@@QAEXII@Z 1000ab18     ZLibInit.obj
 0002:00001b38       __ehfuncinfo$?_Copy@?$basic_string@DU?$char_traits@D@std@@V?$allocator@D@2@@std@@QAEXII@Z 1000ab38     ZLibInit.obj
 0002:00001b5c       __tryblocktable$?_Copy@?$basic_string@DU?$char_traits@D@std@@V?$allocator@D@2@@std@@QAEXII@Z 1000ab5c     ZLibInit.obj
 0002:00001b88       __sehtable$__onexit        1000ab88     MSVCRT:atonexit.obj
 0002:00001ba8       __sehtable$___DllMainCRTStartup 1000aba8     MSVCRT:crtdll.obj
 0002:00001bd0       __sehtable$??_M@YGXPAXIHP6EX0@Z@Z 1000abd0     MSVCRT:ehvecdtr.obj
 0002:00001bf0       __sehtable$?__ArrayUnwind@@YGXPAXIHP6EX0@Z@Z 1000abf0     MSVCRT:ehvecdtr.obj
 0002:00001c10       __sehtable$__IsNonwritableInCurrentImage 1000ac10     MSVCRT:pesect.obj
 0002:00001dd4       .idata$6                   1000add4     kernel32:KERNEL32.dll
 0002:00001e84       .idata$6                   1000ae84     Memory:Memory.dll
 0002:00001f2a       .idata$6                   1000af2a     msvcprt:MSVCP110.dll
 0002:00002076       .idata$6                   1000b076     MSVCRT:MSVCR110.dll
 0002:00002270       .edata                     1000b270     ZLib.exp
 0002:00002298       rgpv                       1000b298     ZLib.exp
 0002:00002354       rgszName                   1000b354     ZLib.exp
 0002:00002410       rgwOrd                     1000b410     ZLib.exp
 0002:0000246e       szName                     1000b46e     ZLib.exp
 0002:00002477       $N00001                    1000b477     ZLib.exp
 0002:0000249d       $N00002                    1000b49d     ZLib.exp
 0002:000024ba       $N00003                    1000b4ba     ZLib.exp
 0002:000024e8       $N00004                    1000b4e8     ZLib.exp
 0002:00002514       $N00005                    1000b514     ZLib.exp
 0002:00002546       $N00006                    1000b546     ZLib.exp
 0002:00002574       $N00007                    1000b574     ZLib.exp
 0002:00002580       $N00008                    1000b580     ZLib.exp
 0002:0000258e       $N00009                    1000b58e     ZLib.exp
 0002:0000259b       $N00010                    1000b59b     ZLib.exp
 0002:000025a5       $N00011                    1000b5a5     ZLib.exp
 0002:000025b0       $N00012                    1000b5b0     ZLib.exp
 0002:000025bf       $N00013                    1000b5bf     ZLib.exp
 0002:000025cd       $N00014                    1000b5cd     ZLib.exp
 0002:000025df       $N00015                    1000b5df     ZLib.exp
 0002:000025f0       $N00016                    1000b5f0     ZLib.exp
 0002:00002602       $N00017                    1000b602     ZLib.exp
 0002:00002612       $N00018                    1000b612     ZLib.exp
 0002:0000262b       $N00019                    1000b62b     ZLib.exp
 0002:0000263c       $N00020                    1000b63c     ZLib.exp
 0002:00002647       $N00021                    1000b647     ZLib.exp
 0002:00002652       $N00022                    1000b652     ZLib.exp
 0002:0000265b       $N00023                    1000b65b     ZLib.exp
 0002:00002666       $N00024                    1000b666     ZLib.exp
 0002:00002671       $N00025                    1000b671     ZLib.exp
 0002:0000267b       $N00026                    1000b67b     ZLib.exp
 0002:00002686       $N00027                    1000b686     ZLib.exp
 0002:00002690       $N00028                    1000b690     ZLib.exp
 0002:00002699       $N00029                    1000b699     ZLib.exp
 0002:000026a3       $N00030                    1000b6a3     ZLib.exp
 0002:000026ad       $N00031                    1000b6ad     ZLib.exp
 0002:000026b8       $N00032                    1000b6b8     ZLib.exp
 0002:000026c4       $N00033                    1000b6c4     ZLib.exp
 0002:000026cf       $N00034                    1000b6cf     ZLib.exp
 0002:000026df       $N00035                    1000b6df     ZLib.exp
 0002:000026e9       $N00036                    1000b6e9     ZLib.exp
 0002:000026f5       $N00037                    1000b6f5     ZLib.exp
 0002:00002700       $N00038                    1000b700     ZLib.exp
 0002:0000270e       $N00039                    1000b70e     ZLib.exp
 0002:00002720       $N00040                    1000b720     ZLib.exp
 0002:00002731       $N00041                    1000b731     ZLib.exp
 0002:00002741       $N00042                    1000b741     ZLib.exp
 0002:0000275a       $N00043                    1000b75a     ZLib.exp
 0002:00002769       $N00044                    1000b769     ZLib.exp
 0002:0000277d       $N00045                    1000b77d     ZLib.exp
 0002:0000278c       $N00046                    1000b78c     ZLib.exp
 0002:00002796       $N00047                    1000b796     ZLib.exp
 0003:000000b4       ?my_version@?1??deflateInit2_@@9@9 1000c0b4     deflate.obj
 0003:000000b8       _gz_magic                  1000c0b8     gzio.obj
 0003:000000c0       _fixed_bl                  1000c0c0     inftrees.obj
 0003:000000c4       _fixed_bd                  1000c0c4     inftrees.obj
 0003:000000c8       _fixed_tl                  1000c0c8     inftrees.obj
 0003:000010c8       _fixed_td                  1000d0c8     inftrees.obj
 0003:0000120c       _static_l_desc             1000d20c     trees.obj
 0003:00001220       _static_d_desc             1000d220     trees.obj
 0003:00001234       _static_bl_desc            1000d234     trees.obj
 0003:000012a0       _allocator_arg             1000d2a0     ZLibInit.obj
 0003:000012a1       _piecewise_construct       1000d2a1     ZLibInit.obj
 0003:000012ac       _allocator_arg             1000d2ac     pch.obj
 0003:000012ad       _piecewise_construct       1000d2ad     pch.obj
 0003:000012ae       _allocator_arg             1000d2ae     Compression1.obj
 0003:000012af       _piecewise_construct       1000d2af     Compression1.obj
 0003:000012b0       _allocator_arg             1000d2b0     CompressionMem1.obj
 0003:000012b1       _piecewise_construct       1000d2b1     CompressionMem1.obj
 0003:000012b4       _s_pool                    1000d2b4     CompressionMem1.obj
 0003:000012b8       ___proc_attached           1000d2b8     MSVCRT:crtdll.obj
 0003:000012c8       _GS_ExceptionRecord        1000d2c8     MSVCRT:gs_report.obj
 0003:00001318       _GS_ContextRecord          1000d318     MSVCRT:gs_report.obj
 0003:000015e4       _DebuggerWasPresent        1000d5e4     MSVCRT:gs_report.obj
 0004:00000060       $R000000                   1000e060     * linker generated manifest res *
